Archive member included because of file (symbol)

c:/program files/microchip/mplab c30/bin/bin/../../lib\libpic30-coff.a(crt1.o)
                              (_resetALT)
c:/program files/microchip/mplab c30/bin/bin/../../lib\libpic30-coff.a(crt0.o)
                              (_resetPRI)
c:/program files/microchip/mplab c30/bin/bin/../../lib\libm-coff.a(divmoddi3.o)
                              ..\Microchip\TCPIP Stack\Objects - TCPIP Demo App-C30\Tick.o (__udivdi3)
c:/program files/microchip/mplab c30/bin/bin/../../lib\libm-coff.a(udivsi3.o)
                              ..\Microchip\TCPIP Stack\Objects - TCPIP Demo App-C30\Helpers.o (__udivsi3)
c:/program files/microchip/mplab c30/bin/bin/../../lib\libc-coff.a(strlen.o)
                              Objects - TCPIP Demo App-C30\MainDemo.o (strlen)
c:/program files/microchip/mplab c30/bin/bin/../../lib\libc-coff.a(memcmp.o)
                              Objects - TCPIP Demo App-C30\CustomHTTPApp.o (memcmp)
c:/program files/microchip/mplab c30/bin/bin/../../lib\libc-coff.a(strcmp.o)
                              Objects - TCPIP Demo App-C30\CustomHTTPApp.o (strcmp)
c:/program files/microchip/mplab c30/bin/bin/../../lib\libc-coff.a(memset.o)
                              ..\Microchip\TCPIP Stack\Objects - TCPIP Demo App-C30\UDP.o (memset)
c:/program files/microchip/mplab c30/bin/bin/../../lib\libc-coff.a(rand.o)
                              ..\Microchip\TCPIP Stack\Objects - TCPIP Demo App-C30\Helpers.o (rand)
c:/program files/microchip/mplab c30/bin/bin/../../lib\libc-coff.a(srand.o)
                              ..\Microchip\TCPIP Stack\Objects - TCPIP Demo App-C30\Helpers.o (srand)
c:/program files/microchip/mplab c30/bin/bin/../../lib\libc-coff.a(xstoul.o)
                              ..\Microchip\TCPIP Stack\Objects - TCPIP Demo App-C30\HTTP2.o (_Stoul)
c:/program files/microchip/mplab c30/bin/bin/../../lib\libc-coff.a(strchr.o)
                              ..\Microchip\TCPIP Stack\Objects - TCPIP Demo App-C30\SMTP.o (strchr)
c:/program files/microchip/mplab c30/bin/bin/../../lib\libc-coff.a(strstr.o)
                              ..\Microchip\TCPIP Stack\Objects - TCPIP Demo App-C30\SMTP.o (strstr)
c:/program files/microchip/mplab c30/bin/bin/../../lib\libc-coff.a(memcpy.o)
                              ..\Microchip\TCPIP Stack\Objects - TCPIP Demo App-C30\TCP.o (memcpy)
c:/program files/microchip/mplab c30/bin/bin/../../lib\libc-coff.a(isspace.os)
                              c:/program files/microchip/mplab c30/bin/bin/../../lib\libc-coff.a(xstoul.o) (isspace)
c:/program files/microchip/mplab c30/bin/bin/../../lib\libc-coff.a(tolower.os)
                              c:/program files/microchip/mplab c30/bin/bin/../../lib\libc-coff.a(xstoul.o) (tolower)
c:/program files/microchip/mplab c30/bin/bin/../../lib\libc-coff.a(memchr.o)
                              c:/program files/microchip/mplab c30/bin/bin/../../lib\libc-coff.a(xstoul.o) (memchr)
c:/program files/microchip/mplab c30/bin/bin/../../lib\libc-coff.a(errno.o)
                              c:/program files/microchip/mplab c30/bin/bin/../../lib\libc-coff.a(xstoul.o) (errno)
c:/program files/microchip/mplab c30/bin/bin/../../lib\libm-coff.a(mulsi3.o)
                              c:/program files/microchip/mplab c30/bin/bin/../../lib\libc-coff.a(rand.o) (__mulsi3)


Program Memory  [Origin = 0x200, Length = 0x155fc]

section                    address   length (PC units)   length (bytes) (dec)
-------                    -------   -----------------   --------------------
.text                        0x200               0x5a0           0x870  (2160)
.const                       0x7a0               0x88e           0xcd5  (3285)
.text                       0x102e              0x20c8          0x312c  (12588)
.text                       0x30f6              0x152a          0x1fbf  (8127)
.text                       0x4620               0xec0          0x1620  (5664)
.text                       0x54e0               0xcb6          0x1311  (4881)
.text                       0x6196               0xb5a          0x1107  (4359)
.text                       0x6cf0               0x964           0xe16  (3606)
.text                       0x7654               0x956           0xe01  (3585)
.text                       0x7faa               0x8d2           0xd3b  (3387)
.text                       0x887c               0x792           0xb5b  (2907)
.text                       0x900e               0x532           0x7cb  (1995)
.text                       0x9540               0x51a           0x7a7  (1959)
.text                       0x9a5a               0x4c4           0x726  (1830)
.text                       0x9f1e               0x3a8           0x57c  (1404)
.text                       0xa2c6               0x386           0x549  (1353)
.text                       0xa64c               0x31e           0x4ad  (1197)
.text                       0xa96a               0x2e2           0x453  (1107)
.text                       0xac4c               0x258           0x384  (900)
.text                       0xaea4               0x1ac           0x282  (642)
.text                       0xb050               0x1a8           0x27c  (636)
.dinit                      0xb1f8               0x198           0x264  (612)
MPFSData                    0xb390               0x110           0x198  (408)
.text                       0xb4a0               0x106           0x189  (393)
.text                       0xb5a6                0xfa           0x177  (375)
.text                       0xb6a0                0x7e            0xbd  (189)
.text                       0xb71e                0x56            0x81  (129)
MPFSHelpers                 0xb774                 0xe            0x15  (21)
.isr                        0xb782                 0x2             0x3  (3)

                     Total program memory used (bytes):        0x11046  (69702) 53%


Data Memory  [Origin = 0x800, Length = 0x2000]

section                    address      alignment gaps    total length  (dec)
-------                    -------      --------------    -------------------
.icd                         0x800                0x50            0x50  (80)
.nbss                        0x850                   0           0x38e  (910)
.ndata                       0xbde                   0            0x90  (144)
.nbss                        0xc6e                   0           0x116  (278)
.ndata                       0xd84                   0            0x22  (34)
.nbss                        0xda6                   0            0x76  (118)
.ndata                       0xe1c                   0             0x6  (6)
.nbss                        0xe22                   0             0x6  (6)
.ndata                       0xe28                   0             0x8  (8)
.nbss                        0xe30                   0             0x8  (8)
.ndata                       0xe38                   0             0x2  (2)
_014c8af04a4a21c5            0xe3a                   0             0x2  (2)
.ndata                       0xe3c                   0             0x2  (2)
_014bfc404a4a21cb            0xe3e                   0             0x2  (2)
.ndata                       0xe40                   0             0x4  (4)
_014d9b604a4a21dc            0xe44                   0             0x2  (2)
.bss                         0xe46                   0            0x88  (136)
.data                        0xece                   0            0x58  (88)

                        Total data memory used (bytes):          0x726  (1830) 22%


Dynamic Memory Usage

region                     address                      maximum length  (dec)
------                     -------                      ---------------------
heap                             0                                   0  (0)
stack                        0xf26                              0x18da  (6362)

                        Maximum dynamic memory (bytes):         0x18da  (6362)


External Symbols in Data Memory (by address):

                    0x09f0                  _UDPSocketInfo
                    0x0a7c                  _activeUDPSocket
                    0x0a7e                  _UDPTxCount
                    0x0a80                  _UDPRxCount
                    0x0a82                  _curHTTP
                    0x0b04                  _httpStubs
                    0x0b0c                  _curHTTPID
                    0x0b7a                  _bufName
                    0x0bac                  _bufFact
                    0x0c72                  _AppConfig
                    0x0ca5                  _AN0String
                    0x0cae                  _lastBlock
                    0x0d18                  _DDNSClient
                    0x0d4a                  _SMTPClient
                    0x0d9e                  _ddnsServiceHosts
                    0x0da6                  _LCDText
                    0x0df8                  _remoteNode
                    0x0e1c                  _smDHCPState
                    0x0e1e                  _DHCPFlags
                    0x0e20                  _DHCPBindCount
                    0x0e28                  _myDHCPBindCount
                    0x0e2a                  ___C30_UART
                    0x0e3c                  _bDHCPServerEnabled
                    0x0f18                  __Tls_setup__Randseed
                    0x0f1a                  __Randseed
                    0x0f1e                  __Tls_setup__Randinit
                    0x0f20                  __Randinit
                    0x0f22                  __Tls_setup_errno
                    0x0f24                  _errno

External Symbols in Data Memory (by name):

                    0x0ca5                  _AN0String
                    0x0c72                  _AppConfig
                    0x0d18                  _DDNSClient
                    0x0e20                  _DHCPBindCount
                    0x0e1e                  _DHCPFlags
                    0x0da6                  _LCDText
                    0x0d4a                  _SMTPClient
                    0x0a80                  _UDPRxCount
                    0x09f0                  _UDPSocketInfo
                    0x0a7e                  _UDPTxCount
                    0x0f20                  __Randinit
                    0x0f1a                  __Randseed
                    0x0f1e                  __Tls_setup__Randinit
                    0x0f18                  __Tls_setup__Randseed
                    0x0f22                  __Tls_setup_errno
                    0x0e2a                  ___C30_UART
                    0x0a7c                  _activeUDPSocket
                    0x0e3c                  _bDHCPServerEnabled
                    0x0bac                  _bufFact
                    0x0b7a                  _bufName
                    0x0a82                  _curHTTP
                    0x0b0c                  _curHTTPID
                    0x0d9e                  _ddnsServiceHosts
                    0x0f24                  _errno
                    0x0b04                  _httpStubs
                    0x0cae                  _lastBlock
                    0x0e28                  _myDHCPBindCount
                    0x0df8                  _remoteNode
                    0x0e1c                  _smDHCPState

External Symbols in Program Memory (by address):

                  0x000200                  __resetPRI
                  0x00021e                  __psv_init
                  0x00022e                  __data_init
                  0x000288                  _strlen
                  0x000296                  _memcmp
                  0x0002b2                  _strcmp
                  0x0002d6                  _memset
                  0x0002e4                  _rand
                  0x00038e                  _srand
                  0x0003b0                  __Stoul
                  0x0004d8                  _strchr
                  0x0004ea                  _strstr
                  0x000512                  _memcpy
                  0x000520                  _isspace
                  0x000530                  _tolower
                  0x00053e                  _memchr
                  0x000552                  __Geterrno
                  0x000584                  ___udivmoddi3
                  0x000652                  ___udivdi3
                  0x000660                  ___umoddi3
                  0x000668                  ___divdi3
                  0x0006a2                  ___moddi3
                  0x000774                  ___udivsi3
                  0x000794                  ___mulsi3
                  0x000fba                  _TCPSocketInitializer
                  0x00102a                  _MPFS_Start
                  0x0010ca                  _TCPInit
                  0x001190                  _TCPOpen
                  0x0012d6                  _TCPWasReset
                  0x0012fa                  _TCPIsConnected
                  0x001316                  _TCPDisconnect
                  0x001398                  _TCPGetRemoteInfo
                  0x0013b4                  _TCPFlush
                  0x0013d0                  _TCPIsPutReady
                  0x00141a                  _TCPPut
                  0x0014a6                  _TCPPutArray
                  0x001574                  _TCPPutString
                  0x001592                  _TCPGetTxFIFOFull
                  0x0015b0                  _TCPDiscard
                  0x0015ce                  _TCPIsGetReady
                  0x001600                  _TCPGet
                  0x00166a                  _TCPGetArray
                  0x001726                  _TCPGetRxFIFOFree
                  0x001742                  _TCPFindArrayEx
                  0x0019c6                  _TCPFindEx
                  0x0019e4                  _TCPTick
                  0x001e52                  _TCPProcess
                  0x002edc                  _TCPAdjustFIFOSize
                  0x0030f6                  _HTTPPrint
                  0x003116                  _HTTPPrint_
                  0x003130                  _HTTPInit
                  0x0031a0                  _HTTPServer
                  0x004246                  _HTTPURLDecode
                  0x00430c                  _HTTPGetArg
                  0x004354                  _HTTPReadPostName
                  0x00437c                  _HTTPReadPostValue
                  0x004558                  _HTTPIncFile
                  0x004620                  _SMTPBeginUsage
                  0x004674                  _SMTPEndUsage
                  0x0046bc                  _SMTPTask
                  0x005218                  _SMTPSendMail
                  0x005220                  _SMTPIsBusy
                  0x005236                  _SMTPIsPutReady
                  0x005252                  _SMTPPut
                  0x0052f2                  _SMTPPutArray
                  0x00532e                  _SMTPPutString
                  0x005364                  _SMTPFlush
                  0x005370                  _SMTPPutDone
                  0x0054e0                  _MACInit
                  0x005600                  _MACIsLinked
                  0x005614                  _MACIsTxReady
                  0x00562c                  _MACDiscardRx
                  0x005660                  _MACGetFreeRxSize
                  0x0056e8                  _MACGetHeader
                  0x0057ca                  _MACPutHeader
                  0x00581e                  _MACFlush
                  0x00593a                  _MACSetReadPtrInRx
                  0x005968                  _MACSetWritePtr
                  0x005996                  _MACSetReadPtr
                  0x0059c4                  _MACCalcRxChecksum
                  0x005a1c                  _CalcIPBufferChecksum
                  0x005ad0                  _MACMemCopyAsync
                  0x005c7e                  _MACIsMemCopyDone
                  0x005c96                  _MACGet
                  0x005cc8                  _MACGetArray
                  0x005da2                  _MACPut
                  0x005dda                  _MACPutArray
                  0x005f96                  _ReadPHYReg
                  0x0060c8                  _WritePHYReg
                  0x006118                  _MACPowerDown
                  0x006146                  _MACPowerUp
                  0x006166                  _SetCLKOUT
                  0x00617c                  _GetCLKOUT
                  0x006196                  _MPFSInit
                  0x0061c0                  _MPFSOpen
                  0x00630e                  _MPFSOpenID
                  0x006392                  _MPFSClose
                  0x0063b4                  _MPFSGet
                  0x00655a                  _MPFSGetArray
                  0x0067be                  _MPFSGetLong
                  0x0067de                  _MPFSSeek
                  0x0069f8                  _MPFSGetTimestamp
                  0x006a46                  _MPFSGetMicrotime
                  0x006a94                  _MPFSGetFlags
                  0x006ad8                  _MPFSGetSize
                  0x006b26                  _MPFSGetBytesRem
                  0x006b6e                  _MPFSGetStartAddr
                  0x006bbe                  _MPFSGetEndAddr
                  0x006c18                  _MPFSGetFilename
                  0x006c80                  _MPFSGetPosition
                  0x006ca0                  _MPFSGetID
                  0x006cf0                  _DDNSInit
                  0x006d32                  _DDNSTask
                  0x00760a                  _DDNSForceUpdate
                  0x007620                  _DDNSSetService
                  0x007640                  _DDNSGetLastIP
                  0x00764c                  _DDNSGetLastStatus
                  0x007654                  _GenerateRandomDWORD
                  0x00776e                  _StringToIPAddress
                  0x0078ee                  _Base64Decode
                  0x007a54                  _Base64Encode
                  0x007bb0                  _uitoa
                  0x007c2e                  _ultoa
                  0x007cde                  _hexatob
                  0x007d54                  _btohexa_high
                  0x007d7c                  _btohexa_low
                  0x007da2                  _stricmppgm2ram
                  0x007e3a                  _swaps
                  0x007e54                  _swapl
                  0x007eb2                  _CalcIPChecksum
                  0x007f28                  _strupr
                  0x007f62                  _FormatNetBIOSName
                  0x007faa                  _DHCPReset
                  0x007fcc                  _DHCPDisable
                  0x007fe8                  _DHCPEnable
                  0x008000                  _DHCPTask
                  0x00887c                  _DNSBeginUsage
                  0x008898                  _DNSEndUsage
                  0x0088be                  _DNSResolve
                  0x0088ee                  _DNSIsResolved
                  0x00900e                  _UDPInit
                  0x009028                  _UDPTask
                  0x009032                  _UDPOpen
                  0x0090c0                  _UDPClose
                  0x0090ea                  _UDPSetTxBuffer
                  0x0090fe                  _UDPSetRxBuffer
                  0x009112                  _UDPIsPutReady
                  0x009148                  _UDPPut
                  0x00917c                  _UDPPutArray
                  0x0091b4                  _UDPPutString
                  0x0091ca                  _UDPFlush
                  0x0092a0                  _UDPIsGetReady
                  0x0092d0                  _UDPGet
                  0x009306                  _UDPGetArray
                  0x009350                  _UDPDiscard
                  0x00936c                  _UDPProcess
                  0x009540                  _DHCPServerTask
                  0x009a5a                  _HashAddData
                  0x009a76                  _MD5Initialize
                  0x009ab2                  _MD5AddData
                  0x009db2                  _MD5Calculate
                  0x009f98                  _ARPInit
                  0x009fce                  _ARPProcess
                  0x00a0ce                  _ARPResolve
                  0x00a19a                  _ARPIsResolved
                  0x00a2c6                  _NBNSTask
                  0x00a64c                  _HTTPNeedsAuth
                  0x00a682                  _HTTPCheckAuth
                  0x00a6b0                  _HTTPExecuteGet
                  0x00a8da                  _HTTPExecutePost
                  0x00a96a                  __AddressError
                  0x00a974                  __StackError
                  0x00a97e                  _main
                  0x00aa22                  _DisplayIPValue
                  0x00ac4c                  _StackInit
                  0x00ac84                  _StackTask
                  0x00ae8a                  _StackApplications
                  0x00aea4                  _IPGetHeader
                  0x00af6e                  _IPPutHeader
                  0x00b00c                  _IPSetRxBuffer
                  0x00b094                  _LCDInit
                  0x00b120                  _LCDUpdate
                  0x00b1dc                  _LCDErase
                  0x00b394                  BEGIN_MPFS
                  0x00b4a0                  _SMTPDemo
                  0x00b5a6                  _TickInit
                  0x00b622                  _TickGet
                  0x00b62e                  _TickGetDiv256
                  0x00b648                  _TickGetDiv64K
                  0x00b662                  _TickConvertToMilliseconds
                  0x00b688                  __T1Interrupt
                  0x00b6a0                  _ICMPProcess
                  0x00b71e                  _DelayMs
                  0x00b748                  _Delay10us
                  0x00b774                  _ReadProgramMemory
                  0x00b782                  __DefaultInterrupt

External Symbols in Program Memory (by name):

                  0x00b394                  BEGIN_MPFS
                  0x009f98                  _ARPInit
                  0x00a19a                  _ARPIsResolved
                  0x009fce                  _ARPProcess
                  0x00a0ce                  _ARPResolve
                  0x0078ee                  _Base64Decode
                  0x007a54                  _Base64Encode
                  0x005a1c                  _CalcIPBufferChecksum
                  0x007eb2                  _CalcIPChecksum
                  0x00760a                  _DDNSForceUpdate
                  0x007640                  _DDNSGetLastIP
                  0x00764c                  _DDNSGetLastStatus
                  0x006cf0                  _DDNSInit
                  0x007620                  _DDNSSetService
                  0x006d32                  _DDNSTask
                  0x007fcc                  _DHCPDisable
                  0x007fe8                  _DHCPEnable
                  0x007faa                  _DHCPReset
                  0x009540                  _DHCPServerTask
                  0x008000                  _DHCPTask
                  0x00887c                  _DNSBeginUsage
                  0x008898                  _DNSEndUsage
                  0x0088ee                  _DNSIsResolved
                  0x0088be                  _DNSResolve
                  0x00b748                  _Delay10us
                  0x00b71e                  _DelayMs
                  0x00aa22                  _DisplayIPValue
                  0x007f62                  _FormatNetBIOSName
                  0x007654                  _GenerateRandomDWORD
                  0x00617c                  _GetCLKOUT
                  0x00a682                  _HTTPCheckAuth
                  0x00a6b0                  _HTTPExecuteGet
                  0x00a8da                  _HTTPExecutePost
                  0x00430c                  _HTTPGetArg
                  0x004558                  _HTTPIncFile
                  0x003130                  _HTTPInit
                  0x00a64c                  _HTTPNeedsAuth
                  0x0030f6                  _HTTPPrint
                  0x003116                  _HTTPPrint_
                  0x004354                  _HTTPReadPostName
                  0x00437c                  _HTTPReadPostValue
                  0x0031a0                  _HTTPServer
                  0x004246                  _HTTPURLDecode
                  0x009a5a                  _HashAddData
                  0x00b6a0                  _ICMPProcess
                  0x00aea4                  _IPGetHeader
                  0x00af6e                  _IPPutHeader
                  0x00b00c                  _IPSetRxBuffer
                  0x00b1dc                  _LCDErase
                  0x00b094                  _LCDInit
                  0x00b120                  _LCDUpdate
                  0x0059c4                  _MACCalcRxChecksum
                  0x00562c                  _MACDiscardRx
                  0x00581e                  _MACFlush
                  0x005c96                  _MACGet
                  0x005cc8                  _MACGetArray
                  0x005660                  _MACGetFreeRxSize
                  0x0056e8                  _MACGetHeader
                  0x0054e0                  _MACInit
                  0x005600                  _MACIsLinked
                  0x005c7e                  _MACIsMemCopyDone
                  0x005614                  _MACIsTxReady
                  0x005ad0                  _MACMemCopyAsync
                  0x006118                  _MACPowerDown
                  0x006146                  _MACPowerUp
                  0x005da2                  _MACPut
                  0x005dda                  _MACPutArray
                  0x0057ca                  _MACPutHeader
                  0x005996                  _MACSetReadPtr
                  0x00593a                  _MACSetReadPtrInRx
                  0x005968                  _MACSetWritePtr
                  0x009ab2                  _MD5AddData
                  0x009db2                  _MD5Calculate
                  0x009a76                  _MD5Initialize
                  0x006392                  _MPFSClose
                  0x0063b4                  _MPFSGet
                  0x00655a                  _MPFSGetArray
                  0x006b26                  _MPFSGetBytesRem
                  0x006bbe                  _MPFSGetEndAddr
                  0x006c18                  _MPFSGetFilename
                  0x006a94                  _MPFSGetFlags
                  0x006ca0                  _MPFSGetID
                  0x0067be                  _MPFSGetLong
                  0x006a46                  _MPFSGetMicrotime
                  0x006c80                  _MPFSGetPosition
                  0x006ad8                  _MPFSGetSize
                  0x006b6e                  _MPFSGetStartAddr
                  0x0069f8                  _MPFSGetTimestamp
                  0x006196                  _MPFSInit
                  0x0061c0                  _MPFSOpen
                  0x00630e                  _MPFSOpenID
                  0x0067de                  _MPFSSeek
                  0x00102a                  _MPFS_Start
                  0x00a2c6                  _NBNSTask
                  0x005f96                  _ReadPHYReg
                  0x00b774                  _ReadProgramMemory
                  0x004620                  _SMTPBeginUsage
                  0x00b4a0                  _SMTPDemo
                  0x004674                  _SMTPEndUsage
                  0x005364                  _SMTPFlush
                  0x005220                  _SMTPIsBusy
                  0x005236                  _SMTPIsPutReady
                  0x005252                  _SMTPPut
                  0x0052f2                  _SMTPPutArray
                  0x005370                  _SMTPPutDone
                  0x00532e                  _SMTPPutString
                  0x005218                  _SMTPSendMail
                  0x0046bc                  _SMTPTask
                  0x006166                  _SetCLKOUT
                  0x00ae8a                  _StackApplications
                  0x00ac4c                  _StackInit
                  0x00ac84                  _StackTask
                  0x00776e                  _StringToIPAddress
                  0x002edc                  _TCPAdjustFIFOSize
                  0x0015b0                  _TCPDiscard
                  0x001316                  _TCPDisconnect
                  0x001742                  _TCPFindArrayEx
                  0x0019c6                  _TCPFindEx
                  0x0013b4                  _TCPFlush
                  0x001600                  _TCPGet
                  0x00166a                  _TCPGetArray
                  0x001398                  _TCPGetRemoteInfo
                  0x001726                  _TCPGetRxFIFOFree
                  0x001592                  _TCPGetTxFIFOFull
                  0x0010ca                  _TCPInit
                  0x0012fa                  _TCPIsConnected
                  0x0015ce                  _TCPIsGetReady
                  0x0013d0                  _TCPIsPutReady
                  0x001190                  _TCPOpen
                  0x001e52                  _TCPProcess
                  0x00141a                  _TCPPut
                  0x0014a6                  _TCPPutArray
                  0x001574                  _TCPPutString
                  0x000fba                  _TCPSocketInitializer
                  0x0019e4                  _TCPTick
                  0x0012d6                  _TCPWasReset
                  0x00b662                  _TickConvertToMilliseconds
                  0x00b622                  _TickGet
                  0x00b62e                  _TickGetDiv256
                  0x00b648                  _TickGetDiv64K
                  0x00b5a6                  _TickInit
                  0x0090c0                  _UDPClose
                  0x009350                  _UDPDiscard
                  0x0091ca                  _UDPFlush
                  0x0092d0                  _UDPGet
                  0x009306                  _UDPGetArray
                  0x00900e                  _UDPInit
                  0x0092a0                  _UDPIsGetReady
                  0x009112                  _UDPIsPutReady
                  0x009032                  _UDPOpen
                  0x00936c                  _UDPProcess
                  0x009148                  _UDPPut
                  0x00917c                  _UDPPutArray
                  0x0091b4                  _UDPPutString
                  0x0090fe                  _UDPSetRxBuffer
                  0x0090ea                  _UDPSetTxBuffer
                  0x009028                  _UDPTask
                  0x0060c8                  _WritePHYReg
                  0x00a96a                  __AddressError
                  0x00b782                  __DefaultInterrupt
                  0x000552                  __Geterrno
                  0x00a974                  __StackError
                  0x0003b0                  __Stoul
                  0x00b688                  __T1Interrupt
                  0x000668                  ___divdi3
                  0x0006a2                  ___moddi3
                  0x000794                  ___mulsi3
                  0x000652                  ___udivdi3
                  0x000584                  ___udivmoddi3
                  0x000774                  ___udivsi3
                  0x000660                  ___umoddi3
                  0x00022e                  __data_init
                  0x00021e                  __psv_init
                  0x000200                  __resetPRI
                  0x007d54                  _btohexa_high
                  0x007d7c                  _btohexa_low
                  0x007cde                  _hexatob
                  0x000520                  _isspace
                  0x00a97e                  _main
                  0x00053e                  _memchr
                  0x000296                  _memcmp
                  0x000512                  _memcpy
                  0x0002d6                  _memset
                  0x0002e4                  _rand
                  0x00038e                  _srand
                  0x0004d8                  _strchr
                  0x0002b2                  _strcmp
                  0x007da2                  _stricmppgm2ram
                  0x000288                  _strlen
                  0x0004ea                  _strstr
                  0x007f28                  _strupr
                  0x007e54                  _swapl
                  0x007e3a                  _swaps
                  0x000530                  _tolower
                  0x007bb0                  _uitoa
                  0x007c2e                  _ultoa

Memory Configuration

Name             Origin             Length             Attributes
data             0x000800           0x002000           a !xr
reset            0x000000           0x000004  
ivt              0x000004           0x0000fc  
aivt             0x000104           0x0000fc  
program          0x000200           0x0155fc           xr
config2          0x0157fc           0x000002  
config1          0x0157fe           0x000002  
*default*        0x000000           0xffffffff  

Linker script and memory map

LOAD Objects - TCPIP Demo App-C30\MainDemo.o
LOAD Objects - TCPIP Demo App-C30\CustomHTTPApp.o
LOAD ..\Microchip\TCPIP Stack\Objects - TCPIP Demo App-C30\Tick.o
LOAD ..\Microchip\TCPIP Stack\Objects - TCPIP Demo App-C30\UART2TCPBridge.o
LOAD ..\Microchip\TCPIP Stack\Objects - TCPIP Demo App-C30\UART.o
LOAD ..\Microchip\TCPIP Stack\Objects - TCPIP Demo App-C30\UDP.o
LOAD ..\Microchip\TCPIP Stack\Objects - TCPIP Demo App-C30\UDPPerformanceTest.o
LOAD ..\Microchip\TCPIP Stack\Objects - TCPIP Demo App-C30\Announce.o
LOAD ..\Microchip\TCPIP Stack\Objects - TCPIP Demo App-C30\ARP.o
LOAD ..\Microchip\TCPIP Stack\Objects - TCPIP Demo App-C30\Delay.o
LOAD ..\Microchip\TCPIP Stack\Objects - TCPIP Demo App-C30\DHCP.o
LOAD ..\Microchip\TCPIP Stack\Objects - TCPIP Demo App-C30\DHCPs.o
LOAD ..\Microchip\TCPIP Stack\Objects - TCPIP Demo App-C30\DNS.o
LOAD ..\Microchip\TCPIP Stack\Objects - TCPIP Demo App-C30\DynDNS.o
LOAD ..\Microchip\TCPIP Stack\Objects - TCPIP Demo App-C30\FTP.o
LOAD ..\Microchip\TCPIP Stack\Objects - TCPIP Demo App-C30\Hashes.o
LOAD ..\Microchip\TCPIP Stack\Objects - TCPIP Demo App-C30\Helpers.o
LOAD ..\Microchip\TCPIP Stack\Objects - TCPIP Demo App-C30\HTTP2.o
LOAD ..\Microchip\TCPIP Stack\Objects - TCPIP Demo App-C30\HTTP.o
LOAD ..\Microchip\TCPIP Stack\Objects - TCPIP Demo App-C30\ICMP.o
LOAD ..\Microchip\TCPIP Stack\Objects - TCPIP Demo App-C30\IP.o
LOAD ..\Microchip\TCPIP Stack\Objects - TCPIP Demo App-C30\LCDBlocking.o
LOAD ..\Microchip\TCPIP Stack\Objects - TCPIP Demo App-C30\MPFS2.o
LOAD ..\Microchip\TCPIP Stack\Objects - TCPIP Demo App-C30\MPFS.o
LOAD ..\Microchip\TCPIP Stack\Objects - TCPIP Demo App-C30\NBNS.o
LOAD ..\Microchip\TCPIP Stack\Objects - TCPIP Demo App-C30\Reboot.o
LOAD ..\Microchip\TCPIP Stack\Objects - TCPIP Demo App-C30\SMTP.o
LOAD ..\Microchip\TCPIP Stack\Objects - TCPIP Demo App-C30\SNMP.o
LOAD ..\Microchip\TCPIP Stack\Objects - TCPIP Demo App-C30\SNTP.o
LOAD ..\Microchip\TCPIP Stack\Objects - TCPIP Demo App-C30\SPIEEPROM.o
LOAD ..\Microchip\TCPIP Stack\Objects - TCPIP Demo App-C30\SPIFlash.o
LOAD ..\Microchip\TCPIP Stack\Objects - TCPIP Demo App-C30\SPIRAM.o
LOAD ..\Microchip\TCPIP Stack\Objects - TCPIP Demo App-C30\StackTsk.o
LOAD ..\Microchip\TCPIP Stack\Objects - TCPIP Demo App-C30\TCP.o
LOAD ..\Microchip\TCPIP Stack\Objects - TCPIP Demo App-C30\TCPPerformanceTest.o
LOAD ..\Microchip\TCPIP Stack\Objects - TCPIP Demo App-C30\Telnet.o
LOAD ..\Microchip\TCPIP Stack\Objects - TCPIP Demo App-C30\TFTPc.o
LOAD Objects - TCPIP Demo App-C30\CustomSNMPApp.o
LOAD Objects - TCPIP Demo App-C30\UARTConfig.o
LOAD Objects - TCPIP Demo App-C30\GenericTCPClient.o
LOAD Objects - TCPIP Demo App-C30\GenericTCPServer.o
LOAD Objects - TCPIP Demo App-C30\PingDemo.o
LOAD Objects - TCPIP Demo App-C30\SMTPDemo.o
LOAD Objects - TCPIP Demo App-C30\LegacyHTTPApp.o
LOAD ..\Microchip\TCPIP Stack\Objects - TCPIP Demo App-C30\BerkeleyAPI.o
LOAD Objects - TCPIP Demo App-C30\BerkeleyUDPClientDemo.o
LOAD Objects - TCPIP Demo App-C30\BerkeleyTCPClientDemo.o
LOAD Objects - TCPIP Demo App-C30\BerkeleyTCPServerDemo.o
LOAD ..\Microchip\TCPIP Stack\Objects - TCPIP Demo App-C30\ENCX24J600.o
LOAD ..\Microchip\TCPIP Stack\Objects - TCPIP Demo App-C30\ENC28J60.o
LOAD Objects - TCPIP Demo App-C30\CustomSSLCert.o
LOAD ..\Microchip\TCPIP Stack\Objects - TCPIP Demo App-C30\SSL.o
LOAD ..\Microchip\TCPIP Stack\Objects - TCPIP Demo App-C30\ARCFOUR.o
LOAD ..\Microchip\TCPIP Stack\Objects - TCPIP Demo App-C30\BigInt.o
LOAD ..\Microchip\TCPIP Stack\Objects - TCPIP Demo App-C30\Random.o
LOAD ..\Microchip\TCPIP Stack\Objects - TCPIP Demo App-C30\RSA.o
LOAD Objects - TCPIP Demo App-C30\MPFSImg2-C30.o
LOAD C:\TCP_Projects\Masters2009\Microchip\TCPIP Stack\BigInt_helper_coff.a
LOAD C:\TCP_Projects\Masters2009\Microchip\TCPIP Stack\BigInt_helper_elf.a
LOAD c:/program files/microchip/mplab c30/bin/bin/../../lib/PIC24F\libpPIC24Fxxx-coff.a
                    0x157fc                  __CONFIG2 = 0x157fc
                    0x157fe                  __CONFIG1 = 0x157fe
                    0x0004                  __IVT_BASE = 0x4
                    0x0104                  __AIVT_BASE = 0x104
                    0x0800                  __DATA_BASE = 0x800
                    0x0200                  __CODE_BASE = 0x200

.reset            0x000000          0x4
                  0x000000          0x2 SHORT 0x200 <code 337> (__reset)
                  0x000001          0x2 SHORT 0x4
                  0x000002          0x2 SHORT 0x0 ((<code 337> (__reset) >> 0x10) & 0x7f)
                  0x000003          0x2 SHORT 0x0

.text             0x000200        0x5a0
 *(.init)
 .init            0x000200         0x88 c:/program files/microchip/mplab c30/bin/bin/../../lib\libpic30-coff.a(crt0.o)
                  0x000200                  _resetPRI
                  0x000200                  _reset
                  0x00021e                  _psv_init
                  0x00022e                  _data_init
 *(.user_init)
 *(.handle)
 *(.libc)
 .libc            0x000288          0xe c:/program files/microchip/mplab c30/bin/bin/../../lib\libc-coff.a(strlen.o)
                  0x000288                  strlen
 .libc            0x000296         0x1c c:/program files/microchip/mplab c30/bin/bin/../../lib\libc-coff.a(memcmp.o)
                  0x000296                  memcmp
 .libc            0x0002b2         0x24 c:/program files/microchip/mplab c30/bin/bin/../../lib\libc-coff.a(strcmp.o)
                  0x0002b2                  strcmp
 .libc            0x0002d6          0xe c:/program files/microchip/mplab c30/bin/bin/../../lib\libc-coff.a(memset.o)
                  0x0002d6                  memset
 .libc            0x0002e4         0xaa c:/program files/microchip/mplab c30/bin/bin/../../lib\libc-coff.a(rand.o)
                  0x0002e4                  rand
 .libc            0x00038e         0x22 c:/program files/microchip/mplab c30/bin/bin/../../lib\libc-coff.a(srand.o)
                  0x00038e                  srand
 .libc            0x0003b0        0x128 c:/program files/microchip/mplab c30/bin/bin/../../lib\libc-coff.a(xstoul.o)
                  0x0003b0                  _Stoul
 .libc            0x0004d8         0x12 c:/program files/microchip/mplab c30/bin/bin/../../lib\libc-coff.a(strchr.o)
                  0x0004d8                  strchr
 .libc            0x0004ea         0x28 c:/program files/microchip/mplab c30/bin/bin/../../lib\libc-coff.a(strstr.o)
                  0x0004ea                  strstr
 .libc            0x000512          0xe c:/program files/microchip/mplab c30/bin/bin/../../lib\libc-coff.a(memcpy.o)
                  0x000512                  memcpy
 .libc            0x000520         0x10 c:/program files/microchip/mplab c30/bin/bin/../../lib\libc-coff.a(isspace.os)
                  0x000520                  isspace
 .libc            0x000530          0xe c:/program files/microchip/mplab c30/bin/bin/../../lib\libc-coff.a(tolower.os)
                  0x000530                  tolower
 .libc            0x00053e         0x14 c:/program files/microchip/mplab c30/bin/bin/../../lib\libc-coff.a(memchr.o)
                  0x00053e                  memchr
 .libc            0x000552          0xc c:/program files/microchip/mplab c30/bin/bin/../../lib\libc-coff.a(errno.o)
                  0x000552                  _Geterrno
 *(.libm)
 .libm            0x00055e        0x216 c:/program files/microchip/mplab c30/bin/bin/../../lib\libm-coff.a(divmoddi3.o)
                  0x000584                  __udivmoddi3
                  0x000652                  __udivdi3
                  0x000660                  __umoddi3
                  0x000668                  __divdi3
                  0x0006a2                  __moddi3
 .libm            0x000774         0x20 c:/program files/microchip/mplab c30/bin/bin/../../lib\libm-coff.a(udivsi3.o)
                  0x000774                  __udivsi3
 .libm            0x000794          0xc c:/program files/microchip/mplab c30/bin/bin/../../lib\libm-coff.a(mulsi3.o)
                  0x000794                  __mulsi3
 *(.libdsp)
 *(.lib*)

__CONFIG2         0x0157fc          0x2
 *(__CONFIG2.sec)
 __CONFIG2.sec    0x0157fc          0x2 Objects - TCPIP Demo App-C30\MainDemo.o

__CONFIG1         0x0157fe          0x2
 *(__CONFIG1.sec)
 __CONFIG1.sec    0x0157fe          0x2 Objects - TCPIP Demo App-C30\MainDemo.o

.icd                0x0800         0x50
                    0x0850                  . = (. + DEFINED (__ICD2RAM)?0x50:0x0)
 *fill*             0x0800         0x5000

.comment
 *(.comment)

.debug_info
 *(.debug_info)
 *(.gnu.linkonce.wi.*)

.debug_abbrev
 *(.debug_abbrev)

.debug_line
 *(.debug_line)

.debug_frame
 *(.debug_frame)

.debug_str
 *(.debug_str)

.debug_loc
 *(.debug_loc)

.debug_macinfo
 *(.debug_macinfo)

.debug_pubnames
 *(.debug_pubnames)

.debug_ranges
 *(.debug_ranges)

.debug_aranges
 *(.debug_aranges)

.ivt              0x000004         0xfc
                  0x000004          0x4 LONG 0xb782 DEFINED (__ReservedTrap0)?<code 337> (__ReservedTrap0):<code 337> (__DefaultInterrupt)
                  0x000006          0x4 LONG 0xb782 DEFINED (__OscillatorFail)?<code 337> (__OscillatorFail):<code 337> (__DefaultInterrupt)
                  0x000008          0x4 LONG 0xa96a DEFINED (__AddressError)?<code 337> (__AddressError):<code 337> (__DefaultInterrupt)
                  0x00000a          0x4 LONG 0xa974 DEFINED (__StackError)?<code 337> (__StackError):<code 337> (__DefaultInterrupt)
                  0x00000c          0x4 LONG 0xb782 DEFINED (__MathError)?<code 337> (__MathError):<code 337> (__DefaultInterrupt)
                  0x00000e          0x4 LONG 0xb782 DEFINED (__ReservedTrap5)?<code 337> (__ReservedTrap5):<code 337> (__DefaultInterrupt)
                  0x000010          0x4 LONG 0xb782 DEFINED (__ReservedTrap6)?<code 337> (__ReservedTrap6):<code 337> (__DefaultInterrupt)
                  0x000012          0x4 LONG 0xb782 DEFINED (__ReservedTrap7)?<code 337> (__ReservedTrap7):<code 337> (__DefaultInterrupt)
                  0x000014          0x4 LONG 0xb782 DEFINED (__INT0Interrupt)?<code 337> (__INT0Interrupt):<code 337> (__DefaultInterrupt)
                  0x000016          0x4 LONG 0xb782 DEFINED (__IC1Interrupt)?<code 337> (__IC1Interrupt):<code 337> (__DefaultInterrupt)
                  0x000018          0x4 LONG 0xb782 DEFINED (__OC1Interrupt)?<code 337> (__OC1Interrupt):<code 337> (__DefaultInterrupt)
                  0x00001a          0x4 LONG 0xb688 DEFINED (__T1Interrupt)?<code 337> (__T1Interrupt):<code 337> (__DefaultInterrupt)
                  0x00001c          0x4 LONG 0xb782 DEFINED (__Interrupt4)?<code 337> (__Interrupt4):<code 337> (__DefaultInterrupt)
                  0x00001e          0x4 LONG 0xb782 DEFINED (__IC2Interrupt)?<code 337> (__IC2Interrupt):<code 337> (__DefaultInterrupt)
                  0x000020          0x4 LONG 0xb782 DEFINED (__OC2Interrupt)?<code 337> (__OC2Interrupt):<code 337> (__DefaultInterrupt)
                  0x000022          0x4 LONG 0xb782 DEFINED (__T2Interrupt)?<code 337> (__T2Interrupt):<code 337> (__DefaultInterrupt)
                  0x000024          0x4 LONG 0xb782 DEFINED (__T3Interrupt)?<code 337> (__T3Interrupt):<code 337> (__DefaultInterrupt)
                  0x000026          0x4 LONG 0xb782 DEFINED (__SPI1ErrInterrupt)?<code 337> (__SPI1ErrInterrupt):<code 337> (__DefaultInterrupt)
                  0x000028          0x4 LONG 0xb782 DEFINED (__SPI1Interrupt)?<code 337> (__SPI1Interrupt):<code 337> (__DefaultInterrupt)
                  0x00002a          0x4 LONG 0xb782 DEFINED (__U1RXInterrupt)?<code 337> (__U1RXInterrupt):<code 337> (__DefaultInterrupt)
                  0x00002c          0x4 LONG 0xb782 DEFINED (__U1TXInterrupt)?<code 337> (__U1TXInterrupt):<code 337> (__DefaultInterrupt)
                  0x00002e          0x4 LONG 0xb782 DEFINED (__ADC1Interrupt)?<code 337> (__ADC1Interrupt):<code 337> (__DefaultInterrupt)
                  0x000030          0x4 LONG 0xb782 DEFINED (__Interrupt14)?<code 337> (__Interrupt14):<code 337> (__DefaultInterrupt)
                  0x000032          0x4 LONG 0xb782 DEFINED (__Interrupt15)?<code 337> (__Interrupt15):<code 337> (__DefaultInterrupt)
                  0x000034          0x4 LONG 0xb782 DEFINED (__SI2C1Interrupt)?<code 337> (__SI2C1Interrupt):<code 337> (__DefaultInterrupt)
                  0x000036          0x4 LONG 0xb782 DEFINED (__MI2C1Interrupt)?<code 337> (__MI2C1Interrupt):<code 337> (__DefaultInterrupt)
                  0x000038          0x4 LONG 0xb782 DEFINED (__CompInterrupt)?<code 337> (__CompInterrupt):<code 337> (__DefaultInterrupt)
                  0x00003a          0x4 LONG 0xb782 DEFINED (__CNInterrupt)?<code 337> (__CNInterrupt):<code 337> (__DefaultInterrupt)
                  0x00003c          0x4 LONG 0xb782 DEFINED (__INT1Interrupt)?<code 337> (__INT1Interrupt):<code 337> (__DefaultInterrupt)
                  0x00003e          0x4 LONG 0xb782 DEFINED (__Interrupt21)?<code 337> (__Interrupt21):<code 337> (__DefaultInterrupt)
                  0x000040          0x4 LONG 0xb782 DEFINED (__Interrupt22)?<code 337> (__Interrupt22):<code 337> (__DefaultInterrupt)
                  0x000042          0x4 LONG 0xb782 DEFINED (__Interrupt23)?<code 337> (__Interrupt23):<code 337> (__DefaultInterrupt)
                  0x000044          0x4 LONG 0xb782 DEFINED (__Interrupt24)?<code 337> (__Interrupt24):<code 337> (__DefaultInterrupt)
                  0x000046          0x4 LONG 0xb782 DEFINED (__OC3Interrupt)?<code 337> (__OC3Interrupt):<code 337> (__DefaultInterrupt)
                  0x000048          0x4 LONG 0xb782 DEFINED (__OC4Interrupt)?<code 337> (__OC4Interrupt):<code 337> (__DefaultInterrupt)
                  0x00004a          0x4 LONG 0xb782 DEFINED (__T4Interrupt)?<code 337> (__T4Interrupt):<code 337> (__DefaultInterrupt)
                  0x00004c          0x4 LONG 0xb782 DEFINED (__T5Interrupt)?<code 337> (__T5Interrupt):<code 337> (__DefaultInterrupt)
                  0x00004e          0x4 LONG 0xb782 DEFINED (__INT2Interrupt)?<code 337> (__INT2Interrupt):<code 337> (__DefaultInterrupt)
                  0x000050          0x4 LONG 0xb782 DEFINED (__U2RXInterrupt)?<code 337> (__U2RXInterrupt):<code 337> (__DefaultInterrupt)
                  0x000052          0x4 LONG 0xb782 DEFINED (__U2TXInterrupt)?<code 337> (__U2TXInterrupt):<code 337> (__DefaultInterrupt)
                  0x000054          0x4 LONG 0xb782 DEFINED (__SPI2ErrInterrupt)?<code 337> (__SPI2ErrInterrupt):<code 337> (__DefaultInterrupt)
                  0x000056          0x4 LONG 0xb782 DEFINED (__SPI2Interrupt)?<code 337> (__SPI2Interrupt):<code 337> (__DefaultInterrupt)
                  0x000058          0x4 LONG 0xb782 DEFINED (__Interrupt34)?<code 337> (__Interrupt34):<code 337> (__DefaultInterrupt)
                  0x00005a          0x4 LONG 0xb782 DEFINED (__Interrupt35)?<code 337> (__Interrupt35):<code 337> (__DefaultInterrupt)
                  0x00005c          0x4 LONG 0xb782 DEFINED (__Interrupt36)?<code 337> (__Interrupt36):<code 337> (__DefaultInterrupt)
                  0x00005e          0x4 LONG 0xb782 DEFINED (__IC3Interrupt)?<code 337> (__IC3Interrupt):<code 337> (__DefaultInterrupt)
                  0x000060          0x4 LONG 0xb782 DEFINED (__IC4Interrupt)?<code 337> (__IC4Interrupt):<code 337> (__DefaultInterrupt)
                  0x000062          0x4 LONG 0xb782 DEFINED (__IC5Interrupt)?<code 337> (__IC5Interrupt):<code 337> (__DefaultInterrupt)
                  0x000064          0x4 LONG 0xb782 DEFINED (__Interrupt40)?<code 337> (__Interrupt40):<code 337> (__DefaultInterrupt)
                  0x000066          0x4 LONG 0xb782 DEFINED (__OC5Interrupt)?<code 337> (__OC5Interrupt):<code 337> (__DefaultInterrupt)
                  0x000068          0x4 LONG 0xb782 DEFINED (__Interrupt42)?<code 337> (__Interrupt42):<code 337> (__DefaultInterrupt)
                  0x00006a          0x4 LONG 0xb782 DEFINED (__Interrupt43)?<code 337> (__Interrupt43):<code 337> (__DefaultInterrupt)
                  0x00006c          0x4 LONG 0xb782 DEFINED (__Interrupt44)?<code 337> (__Interrupt44):<code 337> (__DefaultInterrupt)
                  0x00006e          0x4 LONG 0xb782 DEFINED (__PMPInterrupt)?<code 337> (__PMPInterrupt):<code 337> (__DefaultInterrupt)
                  0x000070          0x4 LONG 0xb782 DEFINED (__Interrupt46)?<code 337> (__Interrupt46):<code 337> (__DefaultInterrupt)
                  0x000072          0x4 LONG 0xb782 DEFINED (__Interrupt47)?<code 337> (__Interrupt47):<code 337> (__DefaultInterrupt)
                  0x000074          0x4 LONG 0xb782 DEFINED (__Interrupt48)?<code 337> (__Interrupt48):<code 337> (__DefaultInterrupt)
                  0x000076          0x4 LONG 0xb782 DEFINED (__SI2C2Interrupt)?<code 337> (__SI2C2Interrupt):<code 337> (__DefaultInterrupt)
                  0x000078          0x4 LONG 0xb782 DEFINED (__MI2C2Interrupt)?<code 337> (__MI2C2Interrupt):<code 337> (__DefaultInterrupt)
                  0x00007a          0x4 LONG 0xb782 DEFINED (__Interrupt51)?<code 337> (__Interrupt51):<code 337> (__DefaultInterrupt)
                  0x00007c          0x4 LONG 0xb782 DEFINED (__Interrupt52)?<code 337> (__Interrupt52):<code 337> (__DefaultInterrupt)
                  0x00007e          0x4 LONG 0xb782 DEFINED (__INT3Interrupt)?<code 337> (__INT3Interrupt):<code 337> (__DefaultInterrupt)
                  0x000080          0x4 LONG 0xb782 DEFINED (__INT4Interrupt)?<code 337> (__INT4Interrupt):<code 337> (__DefaultInterrupt)
                  0x000082          0x4 LONG 0xb782 DEFINED (__Interrupt55)?<code 337> (__Interrupt55):<code 337> (__DefaultInterrupt)
                  0x000084          0x4 LONG 0xb782 DEFINED (__Interrupt56)?<code 337> (__Interrupt56):<code 337> (__DefaultInterrupt)
                  0x000086          0x4 LONG 0xb782 DEFINED (__Interrupt57)?<code 337> (__Interrupt57):<code 337> (__DefaultInterrupt)
                  0x000088          0x4 LONG 0xb782 DEFINED (__Interrupt58)?<code 337> (__Interrupt58):<code 337> (__DefaultInterrupt)
                  0x00008a          0x4 LONG 0xb782 DEFINED (__Interrupt59)?<code 337> (__Interrupt59):<code 337> (__DefaultInterrupt)
                  0x00008c          0x4 LONG 0xb782 DEFINED (__Interrupt60)?<code 337> (__Interrupt60):<code 337> (__DefaultInterrupt)
                  0x00008e          0x4 LONG 0xb782 DEFINED (__Interrupt61)?<code 337> (__Interrupt61):<code 337> (__DefaultInterrupt)
                  0x000090          0x4 LONG 0xb782 DEFINED (__RTCCInterrupt)?<code 337> (__RTCCInterrupt):<code 337> (__DefaultInterrupt)
                  0x000092          0x4 LONG 0xb782 DEFINED (__Interrupt63)?<code 337> (__Interrupt63):<code 337> (__DefaultInterrupt)
                  0x000094          0x4 LONG 0xb782 DEFINED (__Interrupt64)?<code 337> (__Interrupt64):<code 337> (__DefaultInterrupt)
                  0x000096          0x4 LONG 0xb782 DEFINED (__U1ErrInterrupt)?<code 337> (__U1ErrInterrupt):<code 337> (__DefaultInterrupt)
                  0x000098          0x4 LONG 0xb782 DEFINED (__U2ErrInterrupt)?<code 337> (__U2ErrInterrupt):<code 337> (__DefaultInterrupt)
                  0x00009a          0x4 LONG 0xb782 DEFINED (__CRCInterrupt)?<code 337> (__CRCInterrupt):<code 337> (__DefaultInterrupt)
                  0x00009c          0x4 LONG 0xb782 DEFINED (__Interrupt68)?<code 337> (__Interrupt68):<code 337> (__DefaultInterrupt)
                  0x00009e          0x4 LONG 0xb782 DEFINED (__Interrupt69)?<code 337> (__Interrupt69):<code 337> (__DefaultInterrupt)
                  0x0000a0          0x4 LONG 0xb782 DEFINED (__Interrupt70)?<code 337> (__Interrupt70):<code 337> (__DefaultInterrupt)
                  0x0000a2          0x4 LONG 0xb782 DEFINED (__Interrupt71)?<code 337> (__Interrupt71):<code 337> (__DefaultInterrupt)
                  0x0000a4          0x4 LONG 0xb782 DEFINED (__Interrupt72)?<code 337> (__Interrupt72):<code 337> (__DefaultInterrupt)
                  0x0000a6          0x4 LONG 0xb782 DEFINED (__Interrupt73)?<code 337> (__Interrupt73):<code 337> (__DefaultInterrupt)
                  0x0000a8          0x4 LONG 0xb782 DEFINED (__Interrupt74)?<code 337> (__Interrupt74):<code 337> (__DefaultInterrupt)
                  0x0000aa          0x4 LONG 0xb782 DEFINED (__Interrupt75)?<code 337> (__Interrupt75):<code 337> (__DefaultInterrupt)
                  0x0000ac          0x4 LONG 0xb782 DEFINED (__Interrupt76)?<code 337> (__Interrupt76):<code 337> (__DefaultInterrupt)
                  0x0000ae          0x4 LONG 0xb782 DEFINED (__Interrupt77)?<code 337> (__Interrupt77):<code 337> (__DefaultInterrupt)
                  0x0000b0          0x4 LONG 0xb782 DEFINED (__Interrupt78)?<code 337> (__Interrupt78):<code 337> (__DefaultInterrupt)
                  0x0000b2          0x4 LONG 0xb782 DEFINED (__Interrupt79)?<code 337> (__Interrupt79):<code 337> (__DefaultInterrupt)
                  0x0000b4          0x4 LONG 0xb782 DEFINED (__Interrupt80)?<code 337> (__Interrupt80):<code 337> (__DefaultInterrupt)
                  0x0000b6          0x4 LONG 0xb782 DEFINED (__Interrupt81)?<code 337> (__Interrupt81):<code 337> (__DefaultInterrupt)
                  0x0000b8          0x4 LONG 0xb782 DEFINED (__Interrupt82)?<code 337> (__Interrupt82):<code 337> (__DefaultInterrupt)
                  0x0000ba          0x4 LONG 0xb782 DEFINED (__Interrupt83)?<code 337> (__Interrupt83):<code 337> (__DefaultInterrupt)
                  0x0000bc          0x4 LONG 0xb782 DEFINED (__Interrupt84)?<code 337> (__Interrupt84):<code 337> (__DefaultInterrupt)
                  0x0000be          0x4 LONG 0xb782 DEFINED (__Interrupt85)?<code 337> (__Interrupt85):<code 337> (__DefaultInterrupt)
                  0x0000c0          0x4 LONG 0xb782 DEFINED (__Interrupt86)?<code 337> (__Interrupt86):<code 337> (__DefaultInterrupt)
                  0x0000c2          0x4 LONG 0xb782 DEFINED (__Interrupt87)?<code 337> (__Interrupt87):<code 337> (__DefaultInterrupt)
                  0x0000c4          0x4 LONG 0xb782 DEFINED (__Interrupt88)?<code 337> (__Interrupt88):<code 337> (__DefaultInterrupt)
                  0x0000c6          0x4 LONG 0xb782 DEFINED (__Interrupt89)?<code 337> (__Interrupt89):<code 337> (__DefaultInterrupt)
                  0x0000c8          0x4 LONG 0xb782 DEFINED (__Interrupt90)?<code 337> (__Interrupt90):<code 337> (__DefaultInterrupt)
                  0x0000ca          0x4 LONG 0xb782 DEFINED (__Interrupt91)?<code 337> (__Interrupt91):<code 337> (__DefaultInterrupt)
                  0x0000cc          0x4 LONG 0xb782 DEFINED (__Interrupt92)?<code 337> (__Interrupt92):<code 337> (__DefaultInterrupt)
                  0x0000ce          0x4 LONG 0xb782 DEFINED (__Interrupt93)?<code 337> (__Interrupt93):<code 337> (__DefaultInterrupt)
                  0x0000d0          0x4 LONG 0xb782 DEFINED (__Interrupt94)?<code 337> (__Interrupt94):<code 337> (__DefaultInterrupt)
                  0x0000d2          0x4 LONG 0xb782 DEFINED (__Interrupt95)?<code 337> (__Interrupt95):<code 337> (__DefaultInterrupt)
                  0x0000d4          0x4 LONG 0xb782 DEFINED (__Interrupt96)?<code 337> (__Interrupt96):<code 337> (__DefaultInterrupt)
                  0x0000d6          0x4 LONG 0xb782 DEFINED (__Interrupt97)?<code 337> (__Interrupt97):<code 337> (__DefaultInterrupt)
                  0x0000d8          0x4 LONG 0xb782 DEFINED (__Interrupt98)?<code 337> (__Interrupt98):<code 337> (__DefaultInterrupt)
                  0x0000da          0x4 LONG 0xb782 DEFINED (__Interrupt99)?<code 337> (__Interrupt99):<code 337> (__DefaultInterrupt)
                  0x0000dc          0x4 LONG 0xb782 DEFINED (__Interrupt100)?<code 337> (__Interrupt100):<code 337> (__DefaultInterrupt)
                  0x0000de          0x4 LONG 0xb782 DEFINED (__Interrupt101)?<code 337> (__Interrupt101):<code 337> (__DefaultInterrupt)
                  0x0000e0          0x4 LONG 0xb782 DEFINED (__Interrupt102)?<code 337> (__Interrupt102):<code 337> (__DefaultInterrupt)
                  0x0000e2          0x4 LONG 0xb782 DEFINED (__Interrupt103)?<code 337> (__Interrupt103):<code 337> (__DefaultInterrupt)
                  0x0000e4          0x4 LONG 0xb782 DEFINED (__Interrupt104)?<code 337> (__Interrupt104):<code 337> (__DefaultInterrupt)
                  0x0000e6          0x4 LONG 0xb782 DEFINED (__Interrupt105)?<code 337> (__Interrupt105):<code 337> (__DefaultInterrupt)
                  0x0000e8          0x4 LONG 0xb782 DEFINED (__Interrupt106)?<code 337> (__Interrupt106):<code 337> (__DefaultInterrupt)
                  0x0000ea          0x4 LONG 0xb782 DEFINED (__Interrupt107)?<code 337> (__Interrupt107):<code 337> (__DefaultInterrupt)
                  0x0000ec          0x4 LONG 0xb782 DEFINED (__Interrupt108)?<code 337> (__Interrupt108):<code 337> (__DefaultInterrupt)
                  0x0000ee          0x4 LONG 0xb782 DEFINED (__Interrupt109)?<code 337> (__Interrupt109):<code 337> (__DefaultInterrupt)
                  0x0000f0          0x4 LONG 0xb782 DEFINED (__Interrupt110)?<code 337> (__Interrupt110):<code 337> (__DefaultInterrupt)
                  0x0000f2          0x4 LONG 0xb782 DEFINED (__Interrupt111)?<code 337> (__Interrupt111):<code 337> (__DefaultInterrupt)
                  0x0000f4          0x4 LONG 0xb782 DEFINED (__Interrupt112)?<code 337> (__Interrupt112):<code 337> (__DefaultInterrupt)
                  0x0000f6          0x4 LONG 0xb782 DEFINED (__Interrupt113)?<code 337> (__Interrupt113):<code 337> (__DefaultInterrupt)
                  0x0000f8          0x4 LONG 0xb782 DEFINED (__Interrupt114)?<code 337> (__Interrupt114):<code 337> (__DefaultInterrupt)
                  0x0000fa          0x4 LONG 0xb782 DEFINED (__Interrupt115)?<code 337> (__Interrupt115):<code 337> (__DefaultInterrupt)
                  0x0000fc          0x4 LONG 0xb782 DEFINED (__Interrupt116)?<code 337> (__Interrupt116):<code 337> (__DefaultInterrupt)
                  0x0000fe          0x4 LONG 0xb782 DEFINED (__Interrupt117)?<code 337> (__Interrupt117):<code 337> (__DefaultInterrupt)

.aivt             0x000104         0xfc
                  0x000104          0x4 LONG 0xb782 DEFINED (__AltReservedTrap0)?<code 337> (__AltReservedTrap0):DEFINED (__ReservedTrap0)?<code 337> (__ReservedTrap0):<code 337> (__DefaultInterrupt)
                  0x000106          0x4 LONG 0xb782 DEFINED (__AltOscillatorFail)?<code 337> (__AltOscillatorFail):DEFINED (__OscillatorFail)?<code 337> (__OscillatorFail):<code 337> (__DefaultInterrupt)
                  0x000108          0x4 LONG 0xa96a DEFINED (__AltAddressError)?<code 337> (__AltAddressError):DEFINED (__AddressError)?<code 337> (__AddressError):<code 337> (__DefaultInterrupt)
                  0x00010a          0x4 LONG 0xa974 DEFINED (__AltStackError)?<code 337> (__AltStackError):DEFINED (__StackError)?<code 337> (__StackError):<code 337> (__DefaultInterrupt)
                  0x00010c          0x4 LONG 0xb782 DEFINED (__AltMathError)?<code 337> (__AltMathError):DEFINED (__MathError)?<code 337> (__MathError):<code 337> (__DefaultInterrupt)
                  0x00010e          0x4 LONG 0xb782 DEFINED (__AltReservedTrap5)?<code 337> (__AltReservedTrap5):DEFINED (__ReservedTrap5)?<code 337> (__ReservedTrap5):<code 337> (__DefaultInterrupt)
                  0x000110          0x4 LONG 0xb782 DEFINED (__AltReservedTrap6)?<code 337> (__AltReservedTrap6):DEFINED (__ReservedTrap6)?<code 337> (__ReservedTrap6):<code 337> (__DefaultInterrupt)
                  0x000112          0x4 LONG 0xb782 DEFINED (__AltReservedTrap7)?<code 337> (__AltReservedTrap7):DEFINED (__ReservedTrap7)?<code 337> (__ReservedTrap7):<code 337> (__DefaultInterrupt)
                  0x000114          0x4 LONG 0xb782 DEFINED (__AltINT0Interrupt)?<code 337> (__AltINT0Interrupt):DEFINED (__INT0Interrupt)?<code 337> (__INT0Interrupt):<code 337> (__DefaultInterrupt)
                  0x000116          0x4 LONG 0xb782 DEFINED (__AltIC1Interrupt)?<code 337> (__AltIC1Interrupt):DEFINED (__IC1Interrupt)?<code 337> (__IC1Interrupt):<code 337> (__DefaultInterrupt)
                  0x000118          0x4 LONG 0xb782 DEFINED (__AltOC1Interrupt)?<code 337> (__AltOC1Interrupt):DEFINED (__OC1Interrupt)?<code 337> (__OC1Interrupt):<code 337> (__DefaultInterrupt)
                  0x00011a          0x4 LONG 0xb688 DEFINED (__AltT1Interrupt)?<code 337> (__AltT1Interrupt):DEFINED (__T1Interrupt)?<code 337> (__T1Interrupt):<code 337> (__DefaultInterrupt)
                  0x00011c          0x4 LONG 0xb782 DEFINED (__AltInterrupt4)?<code 337> (__AltInterrupt4):DEFINED (__Interrupt4)?<code 337> (__Interrupt4):<code 337> (__DefaultInterrupt)
                  0x00011e          0x4 LONG 0xb782 DEFINED (__AltIC2Interrupt)?<code 337> (__AltIC2Interrupt):DEFINED (__IC2Interrupt)?<code 337> (__IC2Interrupt):<code 337> (__DefaultInterrupt)
                  0x000120          0x4 LONG 0xb782 DEFINED (__AltOC2Interrupt)?<code 337> (__AltOC2Interrupt):DEFINED (__OC2Interrupt)?<code 337> (__OC2Interrupt):<code 337> (__DefaultInterrupt)
                  0x000122          0x4 LONG 0xb782 DEFINED (__AltT2Interrupt)?<code 337> (__AltT2Interrupt):DEFINED (__T2Interrupt)?<code 337> (__T2Interrupt):<code 337> (__DefaultInterrupt)
                  0x000124          0x4 LONG 0xb782 DEFINED (__AltT3Interrupt)?<code 337> (__AltT3Interrupt):DEFINED (__T3Interrupt)?<code 337> (__T3Interrupt):<code 337> (__DefaultInterrupt)
                  0x000126          0x4 LONG 0xb782 DEFINED (__AltSPI1ErrInterrupt)?<code 337> (__AltSPI1ErrInterrupt):DEFINED (__SPI1ErrInterrupt)?<code 337> (__SPI1ErrInterrupt):<code 337> (__DefaultInterrupt)
                  0x000128          0x4 LONG 0xb782 DEFINED (__AltSPI1Interrupt)?<code 337> (__AltSPI1Interrupt):DEFINED (__SPI1Interrupt)?<code 337> (__SPI1Interrupt):<code 337> (__DefaultInterrupt)
                  0x00012a          0x4 LONG 0xb782 DEFINED (__AltU1RXInterrupt)?<code 337> (__AltU1RXInterrupt):DEFINED (__U1RXInterrupt)?<code 337> (__U1RXInterrupt):<code 337> (__DefaultInterrupt)
                  0x00012c          0x4 LONG 0xb782 DEFINED (__AltU1TXInterrupt)?<code 337> (__AltU1TXInterrupt):DEFINED (__U1TXInterrupt)?<code 337> (__U1TXInterrupt):<code 337> (__DefaultInterrupt)
                  0x00012e          0x4 LONG 0xb782 DEFINED (__AltADC1Interrupt)?<code 337> (__AltADC1Interrupt):DEFINED (__ADC1Interrupt)?<code 337> (__ADC1Interrupt):<code 337> (__DefaultInterrupt)
                  0x000130          0x4 LONG 0xb782 DEFINED (__AltInterrupt14)?<code 337> (__AltInterrupt14):DEFINED (__Interrupt14)?<code 337> (__Interrupt14):<code 337> (__DefaultInterrupt)
                  0x000132          0x4 LONG 0xb782 DEFINED (__AltInterrupt15)?<code 337> (__AltInterrupt15):DEFINED (__Interrupt15)?<code 337> (__Interrupt15):<code 337> (__DefaultInterrupt)
                  0x000134          0x4 LONG 0xb782 DEFINED (__AltSI2C1Interrupt)?<code 337> (__AltSI2C1Interrupt):DEFINED (__SI2C1Interrupt)?<code 337> (__SI2C1Interrupt):<code 337> (__DefaultInterrupt)
                  0x000136          0x4 LONG 0xb782 DEFINED (__AltMI2C1Interrupt)?<code 337> (__AltMI2C1Interrupt):DEFINED (__MI2C1Interrupt)?<code 337> (__MI2C1Interrupt):<code 337> (__DefaultInterrupt)
                  0x000138          0x4 LONG 0xb782 DEFINED (__AltCompInterrupt)?<code 337> (__AltCompInterrupt):DEFINED (__CompInterrupt)?<code 337> (__CompInterrupt):<code 337> (__DefaultInterrupt)
                  0x00013a          0x4 LONG 0xb782 DEFINED (__AltCNInterrupt)?<code 337> (__AltCNInterrupt):DEFINED (__CNInterrupt)?<code 337> (__CNInterrupt):<code 337> (__DefaultInterrupt)
                  0x00013c          0x4 LONG 0xb782 DEFINED (__AltINT1Interrupt)?<code 337> (__AltINT1Interrupt):DEFINED (__INT1Interrupt)?<code 337> (__INT1Interrupt):<code 337> (__DefaultInterrupt)
                  0x00013e          0x4 LONG 0xb782 DEFINED (__AltInterrupt21)?<code 337> (__AltInterrupt21):DEFINED (__Interrupt21)?<code 337> (__Interrupt21):<code 337> (__DefaultInterrupt)
                  0x000140          0x4 LONG 0xb782 DEFINED (__AltInterrupt22)?<code 337> (__AltInterrupt22):DEFINED (__Interrupt22)?<code 337> (__Interrupt22):<code 337> (__DefaultInterrupt)
                  0x000142          0x4 LONG 0xb782 DEFINED (__AltInterrupt23)?<code 337> (__AltInterrupt23):DEFINED (__Interrupt23)?<code 337> (__Interrupt23):<code 337> (__DefaultInterrupt)
                  0x000144          0x4 LONG 0xb782 DEFINED (__AltInterrupt24)?<code 337> (__AltInterrupt24):DEFINED (__Interrupt24)?<code 337> (__Interrupt24):<code 337> (__DefaultInterrupt)
                  0x000146          0x4 LONG 0xb782 DEFINED (__AltOC3Interrupt)?<code 337> (__AltOC3Interrupt):DEFINED (__OC3Interrupt)?<code 337> (__OC3Interrupt):<code 337> (__DefaultInterrupt)
                  0x000148          0x4 LONG 0xb782 DEFINED (__AltOC4Interrupt)?<code 337> (__AltOC4Interrupt):DEFINED (__OC4Interrupt)?<code 337> (__OC4Interrupt):<code 337> (__DefaultInterrupt)
                  0x00014a          0x4 LONG 0xb782 DEFINED (__AltT4Interrupt)?<code 337> (__AltT4Interrupt):DEFINED (__T4Interrupt)?<code 337> (__T4Interrupt):<code 337> (__DefaultInterrupt)
                  0x00014c          0x4 LONG 0xb782 DEFINED (__AltT5Interrupt)?<code 337> (__AltT5Interrupt):DEFINED (__T5Interrupt)?<code 337> (__T5Interrupt):<code 337> (__DefaultInterrupt)
                  0x00014e          0x4 LONG 0xb782 DEFINED (__AltINT2Interrupt)?<code 337> (__AltINT2Interrupt):DEFINED (__INT2Interrupt)?<code 337> (__INT2Interrupt):<code 337> (__DefaultInterrupt)
                  0x000150          0x4 LONG 0xb782 DEFINED (__AltU2RXInterrupt)?<code 337> (__AltU2RXInterrupt):DEFINED (__U2RXInterrupt)?<code 337> (__U2RXInterrupt):<code 337> (__DefaultInterrupt)
                  0x000152          0x4 LONG 0xb782 DEFINED (__AltU2TXInterrupt)?<code 337> (__AltU2TXInterrupt):DEFINED (__U2TXInterrupt)?<code 337> (__U2TXInterrupt):<code 337> (__DefaultInterrupt)
                  0x000154          0x4 LONG 0xb782 DEFINED (__AltSPI2ErrInterrupt)?<code 337> (__AltSPI2ErrInterrupt):DEFINED (__SPI2ErrInterrupt)?<code 337> (__SPI2ErrInterrupt):<code 337> (__DefaultInterrupt)
                  0x000156          0x4 LONG 0xb782 DEFINED (__AltSPI2Interrupt)?<code 337> (__AltSPI2Interrupt):DEFINED (__SPI2Interrupt)?<code 337> (__SPI2Interrupt):<code 337> (__DefaultInterrupt)
                  0x000158          0x4 LONG 0xb782 DEFINED (__AltInterrupt34)?<code 337> (__AltInterrupt34):DEFINED (__Interrupt34)?<code 337> (__Interrupt34):<code 337> (__DefaultInterrupt)
                  0x00015a          0x4 LONG 0xb782 DEFINED (__AltInterrupt35)?<code 337> (__AltInterrupt35):DEFINED (__Interrupt35)?<code 337> (__Interrupt35):<code 337> (__DefaultInterrupt)
                  0x00015c          0x4 LONG 0xb782 DEFINED (__AltInterrupt36)?<code 337> (__AltInterrupt36):DEFINED (__Interrupt36)?<code 337> (__Interrupt36):<code 337> (__DefaultInterrupt)
                  0x00015e          0x4 LONG 0xb782 DEFINED (__AltIC3Interrupt)?<code 337> (__AltIC3Interrupt):DEFINED (__IC3Interrupt)?<code 337> (__IC3Interrupt):<code 337> (__DefaultInterrupt)
                  0x000160          0x4 LONG 0xb782 DEFINED (__AltIC4Interrupt)?<code 337> (__AltIC4Interrupt):DEFINED (__IC4Interrupt)?<code 337> (__IC4Interrupt):<code 337> (__DefaultInterrupt)
                  0x000162          0x4 LONG 0xb782 DEFINED (__AltIC5Interrupt)?<code 337> (__AltIC5Interrupt):DEFINED (__IC5Interrupt)?<code 337> (__IC5Interrupt):<code 337> (__DefaultInterrupt)
                  0x000164          0x4 LONG 0xb782 DEFINED (__AltInterrupt40)?<code 337> (__AltInterrupt40):DEFINED (__Interrupt40)?<code 337> (__Interrupt40):<code 337> (__DefaultInterrupt)
                  0x000166          0x4 LONG 0xb782 DEFINED (__AltOC5Interrupt)?<code 337> (__AltOC5Interrupt):DEFINED (__OC5Interrupt)?<code 337> (__OC5Interrupt):<code 337> (__DefaultInterrupt)
                  0x000168          0x4 LONG 0xb782 DEFINED (__AltInterrupt42)?<code 337> (__AltInterrupt42):DEFINED (__Interrupt42)?<code 337> (__Interrupt42):<code 337> (__DefaultInterrupt)
                  0x00016a          0x4 LONG 0xb782 DEFINED (__AltInterrupt43)?<code 337> (__AltInterrupt43):DEFINED (__Interrupt43)?<code 337> (__Interrupt43):<code 337> (__DefaultInterrupt)
                  0x00016c          0x4 LONG 0xb782 DEFINED (__AltInterrupt44)?<code 337> (__AltInterrupt44):DEFINED (__Interrupt44)?<code 337> (__Interrupt44):<code 337> (__DefaultInterrupt)
                  0x00016e          0x4 LONG 0xb782 DEFINED (__AltPMPInterrupt)?<code 337> (__AltPMPInterrupt):DEFINED (__PMPInterrupt)?<code 337> (__PMPInterrupt):<code 337> (__DefaultInterrupt)
                  0x000170          0x4 LONG 0xb782 DEFINED (__AltInterrupt46)?<code 337> (__AltInterrupt46):DEFINED (__Interrupt46)?<code 337> (__Interrupt46):<code 337> (__DefaultInterrupt)
                  0x000172          0x4 LONG 0xb782 DEFINED (__AltInterrupt47)?<code 337> (__AltInterrupt47):DEFINED (__Interrupt47)?<code 337> (__Interrupt47):<code 337> (__DefaultInterrupt)
                  0x000174          0x4 LONG 0xb782 DEFINED (__AltInterrupt48)?<code 337> (__AltInterrupt48):DEFINED (__Interrupt48)?<code 337> (__Interrupt48):<code 337> (__DefaultInterrupt)
                  0x000176          0x4 LONG 0xb782 DEFINED (__AltSI2C2Interrupt)?<code 337> (__AltSI2C2Interrupt):DEFINED (__SI2C2Interrupt)?<code 337> (__SI2C2Interrupt):<code 337> (__DefaultInterrupt)
                  0x000178          0x4 LONG 0xb782 DEFINED (__AltMI2C2Interrupt)?<code 337> (__AltMI2C2Interrupt):DEFINED (__MI2C2Interrupt)?<code 337> (__MI2C2Interrupt):<code 337> (__DefaultInterrupt)
                  0x00017a          0x4 LONG 0xb782 DEFINED (__AltInterrupt51)?<code 337> (__AltInterrupt51):DEFINED (__Interrupt51)?<code 337> (__Interrupt51):<code 337> (__DefaultInterrupt)
                  0x00017c          0x4 LONG 0xb782 DEFINED (__AltInterrupt52)?<code 337> (__AltInterrupt52):DEFINED (__Interrupt52)?<code 337> (__Interrupt52):<code 337> (__DefaultInterrupt)
                  0x00017e          0x4 LONG 0xb782 DEFINED (__AltINT3Interrupt)?<code 337> (__AltINT3Interrupt):DEFINED (__INT3Interrupt)?<code 337> (__INT3Interrupt):<code 337> (__DefaultInterrupt)
                  0x000180          0x4 LONG 0xb782 DEFINED (__AltINT4Interrupt)?<code 337> (__AltINT4Interrupt):DEFINED (__INT4Interrupt)?<code 337> (__INT4Interrupt):<code 337> (__DefaultInterrupt)
                  0x000182          0x4 LONG 0xb782 DEFINED (__AltInterrupt55)?<code 337> (__AltInterrupt55):DEFINED (__Interrupt55)?<code 337> (__Interrupt55):<code 337> (__DefaultInterrupt)
                  0x000184          0x4 LONG 0xb782 DEFINED (__AltInterrupt56)?<code 337> (__AltInterrupt56):DEFINED (__Interrupt56)?<code 337> (__Interrupt56):<code 337> (__DefaultInterrupt)
                  0x000186          0x4 LONG 0xb782 DEFINED (__AltInterrupt57)?<code 337> (__AltInterrupt57):DEFINED (__Interrupt57)?<code 337> (__Interrupt57):<code 337> (__DefaultInterrupt)
                  0x000188          0x4 LONG 0xb782 DEFINED (__AltInterrupt58)?<code 337> (__AltInterrupt58):DEFINED (__Interrupt58)?<code 337> (__Interrupt58):<code 337> (__DefaultInterrupt)
                  0x00018a          0x4 LONG 0xb782 DEFINED (__AltInterrupt59)?<code 337> (__AltInterrupt59):DEFINED (__Interrupt59)?<code 337> (__Interrupt59):<code 337> (__DefaultInterrupt)
                  0x00018c          0x4 LONG 0xb782 DEFINED (__AltInterrupt60)?<code 337> (__AltInterrupt60):DEFINED (__Interrupt60)?<code 337> (__Interrupt60):<code 337> (__DefaultInterrupt)
                  0x00018e          0x4 LONG 0xb782 DEFINED (__AltInterrupt61)?<code 337> (__AltInterrupt61):DEFINED (__Interrupt61)?<code 337> (__Interrupt61):<code 337> (__DefaultInterrupt)
                  0x000190          0x4 LONG 0xb782 DEFINED (__AltRTCCInterrupt)?<code 337> (__AltRTCCInterrupt):DEFINED (__RTCCInterrupt)?<code 337> (__RTCCInterrupt):<code 337> (__DefaultInterrupt)
                  0x000192          0x4 LONG 0xb782 DEFINED (__AltInterrupt63)?<code 337> (__AltInterrupt63):DEFINED (__Interrupt63)?<code 337> (__Interrupt63):<code 337> (__DefaultInterrupt)
                  0x000194          0x4 LONG 0xb782 DEFINED (__AltInterrupt64)?<code 337> (__AltInterrupt64):DEFINED (__Interrupt64)?<code 337> (__Interrupt64):<code 337> (__DefaultInterrupt)
                  0x000196          0x4 LONG 0xb782 DEFINED (__AltU1ErrInterrupt)?<code 337> (__AltU1ErrInterrupt):DEFINED (__U1ErrInterrupt)?<code 337> (__U1ErrInterrupt):<code 337> (__DefaultInterrupt)
                  0x000198          0x4 LONG 0xb782 DEFINED (__AltU2ErrInterrupt)?<code 337> (__AltU2ErrInterrupt):DEFINED (__U2ErrInterrupt)?<code 337> (__U2ErrInterrupt):<code 337> (__DefaultInterrupt)
                  0x00019a          0x4 LONG 0xb782 DEFINED (__AltCRCInterrupt)?<code 337> (__AltCRCInterrupt):DEFINED (__CRCInterrupt)?<code 337> (__CRCInterrupt):<code 337> (__DefaultInterrupt)
                  0x00019c          0x4 LONG 0xb782 DEFINED (__AltInterrupt68)?<code 337> (__AltInterrupt68):DEFINED (__Interrupt68)?<code 337> (__Interrupt68):<code 337> (__DefaultInterrupt)
                  0x00019e          0x4 LONG 0xb782 DEFINED (__AltInterrupt69)?<code 337> (__AltInterrupt69):DEFINED (__Interrupt69)?<code 337> (__Interrupt69):<code 337> (__DefaultInterrupt)
                  0x0001a0          0x4 LONG 0xb782 DEFINED (__AltInterrupt70)?<code 337> (__AltInterrupt70):DEFINED (__Interrupt70)?<code 337> (__Interrupt70):<code 337> (__DefaultInterrupt)
                  0x0001a2          0x4 LONG 0xb782 DEFINED (__AltInterrupt71)?<code 337> (__AltInterrupt71):DEFINED (__Interrupt71)?<code 337> (__Interrupt71):<code 337> (__DefaultInterrupt)
                  0x0001a4          0x4 LONG 0xb782 DEFINED (__AltInterrupt72)?<code 337> (__AltInterrupt72):DEFINED (__Interrupt72)?<code 337> (__Interrupt72):<code 337> (__DefaultInterrupt)
                  0x0001a6          0x4 LONG 0xb782 DEFINED (__AltInterrupt73)?<code 337> (__AltInterrupt73):DEFINED (__Interrupt73)?<code 337> (__Interrupt73):<code 337> (__DefaultInterrupt)
                  0x0001a8          0x4 LONG 0xb782 DEFINED (__AltInterrupt74)?<code 337> (__AltInterrupt74):DEFINED (__Interrupt74)?<code 337> (__Interrupt74):<code 337> (__DefaultInterrupt)
                  0x0001aa          0x4 LONG 0xb782 DEFINED (__AltInterrupt75)?<code 337> (__AltInterrupt75):DEFINED (__Interrupt75)?<code 337> (__Interrupt75):<code 337> (__DefaultInterrupt)
                  0x0001ac          0x4 LONG 0xb782 DEFINED (__AltInterrupt76)?<code 337> (__AltInterrupt76):DEFINED (__Interrupt76)?<code 337> (__Interrupt76):<code 337> (__DefaultInterrupt)
                  0x0001ae          0x4 LONG 0xb782 DEFINED (__AltInterrupt77)?<code 337> (__AltInterrupt77):DEFINED (__Interrupt77)?<code 337> (__Interrupt77):<code 337> (__DefaultInterrupt)
                  0x0001b0          0x4 LONG 0xb782 DEFINED (__AltInterrupt78)?<code 337> (__AltInterrupt78):DEFINED (__Interrupt78)?<code 337> (__Interrupt78):<code 337> (__DefaultInterrupt)
                  0x0001b2          0x4 LONG 0xb782 DEFINED (__AltInterrupt79)?<code 337> (__AltInterrupt79):DEFINED (__Interrupt79)?<code 337> (__Interrupt79):<code 337> (__DefaultInterrupt)
                  0x0001b4          0x4 LONG 0xb782 DEFINED (__AltInterrupt80)?<code 337> (__AltInterrupt80):DEFINED (__Interrupt80)?<code 337> (__Interrupt80):<code 337> (__DefaultInterrupt)
                  0x0001b6          0x4 LONG 0xb782 DEFINED (__AltInterrupt81)?<code 337> (__AltInterrupt81):DEFINED (__Interrupt81)?<code 337> (__Interrupt81):<code 337> (__DefaultInterrupt)
                  0x0001b8          0x4 LONG 0xb782 DEFINED (__AltInterrupt82)?<code 337> (__AltInterrupt82):DEFINED (__Interrupt82)?<code 337> (__Interrupt82):<code 337> (__DefaultInterrupt)
                  0x0001ba          0x4 LONG 0xb782 DEFINED (__AltInterrupt83)?<code 337> (__AltInterrupt83):DEFINED (__Interrupt83)?<code 337> (__Interrupt83):<code 337> (__DefaultInterrupt)
                  0x0001bc          0x4 LONG 0xb782 DEFINED (__AltInterrupt84)?<code 337> (__AltInterrupt84):DEFINED (__Interrupt84)?<code 337> (__Interrupt84):<code 337> (__DefaultInterrupt)
                  0x0001be          0x4 LONG 0xb782 DEFINED (__AltInterrupt85)?<code 337> (__AltInterrupt85):DEFINED (__Interrupt85)?<code 337> (__Interrupt85):<code 337> (__DefaultInterrupt)
                  0x0001c0          0x4 LONG 0xb782 DEFINED (__AltInterrupt86)?<code 337> (__AltInterrupt86):DEFINED (__Interrupt86)?<code 337> (__Interrupt86):<code 337> (__DefaultInterrupt)
                  0x0001c2          0x4 LONG 0xb782 DEFINED (__AltInterrupt87)?<code 337> (__AltInterrupt87):DEFINED (__Interrupt87)?<code 337> (__Interrupt87):<code 337> (__DefaultInterrupt)
                  0x0001c4          0x4 LONG 0xb782 DEFINED (__AltInterrupt88)?<code 337> (__AltInterrupt88):DEFINED (__Interrupt88)?<code 337> (__Interrupt88):<code 337> (__DefaultInterrupt)
                  0x0001c6          0x4 LONG 0xb782 DEFINED (__AltInterrupt89)?<code 337> (__AltInterrupt89):DEFINED (__Interrupt89)?<code 337> (__Interrupt89):<code 337> (__DefaultInterrupt)
                  0x0001c8          0x4 LONG 0xb782 DEFINED (__AltInterrupt90)?<code 337> (__AltInterrupt90):DEFINED (__Interrupt90)?<code 337> (__Interrupt90):<code 337> (__DefaultInterrupt)
                  0x0001ca          0x4 LONG 0xb782 DEFINED (__AltInterrupt91)?<code 337> (__AltInterrupt91):DEFINED (__Interrupt91)?<code 337> (__Interrupt91):<code 337> (__DefaultInterrupt)
                  0x0001cc          0x4 LONG 0xb782 DEFINED (__AltInterrupt92)?<code 337> (__AltInterrupt92):DEFINED (__Interrupt92)?<code 337> (__Interrupt92):<code 337> (__DefaultInterrupt)
                  0x0001ce          0x4 LONG 0xb782 DEFINED (__AltInterrupt93)?<code 337> (__AltInterrupt93):DEFINED (__Interrupt93)?<code 337> (__Interrupt93):<code 337> (__DefaultInterrupt)
                  0x0001d0          0x4 LONG 0xb782 DEFINED (__AltInterrupt94)?<code 337> (__AltInterrupt94):DEFINED (__Interrupt94)?<code 337> (__Interrupt94):<code 337> (__DefaultInterrupt)
                  0x0001d2          0x4 LONG 0xb782 DEFINED (__AltInterrupt95)?<code 337> (__AltInterrupt95):DEFINED (__Interrupt95)?<code 337> (__Interrupt95):<code 337> (__DefaultInterrupt)
                  0x0001d4          0x4 LONG 0xb782 DEFINED (__AltInterrupt96)?<code 337> (__AltInterrupt96):DEFINED (__Interrupt96)?<code 337> (__Interrupt96):<code 337> (__DefaultInterrupt)
                  0x0001d6          0x4 LONG 0xb782 DEFINED (__AltInterrupt97)?<code 337> (__AltInterrupt97):DEFINED (__Interrupt97)?<code 337> (__Interrupt97):<code 337> (__DefaultInterrupt)
                  0x0001d8          0x4 LONG 0xb782 DEFINED (__AltInterrupt98)?<code 337> (__AltInterrupt98):DEFINED (__Interrupt98)?<code 337> (__Interrupt98):<code 337> (__DefaultInterrupt)
                  0x0001da          0x4 LONG 0xb782 DEFINED (__AltInterrupt99)?<code 337> (__AltInterrupt99):DEFINED (__Interrupt99)?<code 337> (__Interrupt99):<code 337> (__DefaultInterrupt)
                  0x0001dc          0x4 LONG 0xb782 DEFINED (__AltInterrupt100)?<code 337> (__AltInterrupt100):DEFINED (__Interrupt100)?<code 337> (__Interrupt100):<code 337> (__DefaultInterrupt)
                  0x0001de          0x4 LONG 0xb782 DEFINED (__AltInterrupt101)?<code 337> (__AltInterrupt101):DEFINED (__Interrupt101)?<code 337> (__Interrupt101):<code 337> (__DefaultInterrupt)
                  0x0001e0          0x4 LONG 0xb782 DEFINED (__AltInterrupt102)?<code 337> (__AltInterrupt102):DEFINED (__Interrupt102)?<code 337> (__Interrupt102):<code 337> (__DefaultInterrupt)
                  0x0001e2          0x4 LONG 0xb782 DEFINED (__AltInterrupt103)?<code 337> (__AltInterrupt103):DEFINED (__Interrupt103)?<code 337> (__Interrupt103):<code 337> (__DefaultInterrupt)
                  0x0001e4          0x4 LONG 0xb782 DEFINED (__AltInterrupt104)?<code 337> (__AltInterrupt104):DEFINED (__Interrupt104)?<code 337> (__Interrupt104):<code 337> (__DefaultInterrupt)
                  0x0001e6          0x4 LONG 0xb782 DEFINED (__AltInterrupt105)?<code 337> (__AltInterrupt105):DEFINED (__Interrupt105)?<code 337> (__Interrupt105):<code 337> (__DefaultInterrupt)
                  0x0001e8          0x4 LONG 0xb782 DEFINED (__AltInterrupt106)?<code 337> (__AltInterrupt106):DEFINED (__Interrupt106)?<code 337> (__Interrupt106):<code 337> (__DefaultInterrupt)
                  0x0001ea          0x4 LONG 0xb782 DEFINED (__AltInterrupt107)?<code 337> (__AltInterrupt107):DEFINED (__Interrupt107)?<code 337> (__Interrupt107):<code 337> (__DefaultInterrupt)
                  0x0001ec          0x4 LONG 0xb782 DEFINED (__AltInterrupt108)?<code 337> (__AltInterrupt108):DEFINED (__Interrupt108)?<code 337> (__Interrupt108):<code 337> (__DefaultInterrupt)
                  0x0001ee          0x4 LONG 0xb782 DEFINED (__AltInterrupt109)?<code 337> (__AltInterrupt109):DEFINED (__Interrupt109)?<code 337> (__Interrupt109):<code 337> (__DefaultInterrupt)
                  0x0001f0          0x4 LONG 0xb782 DEFINED (__AltInterrupt110)?<code 337> (__AltInterrupt110):DEFINED (__Interrupt110)?<code 337> (__Interrupt110):<code 337> (__DefaultInterrupt)
                  0x0001f2          0x4 LONG 0xb782 DEFINED (__AltInterrupt111)?<code 337> (__AltInterrupt111):DEFINED (__Interrupt111)?<code 337> (__Interrupt111):<code 337> (__DefaultInterrupt)
                  0x0001f4          0x4 LONG 0xb782 DEFINED (__AltInterrupt112)?<code 337> (__AltInterrupt112):DEFINED (__Interrupt112)?<code 337> (__Interrupt112):<code 337> (__DefaultInterrupt)
                  0x0001f6          0x4 LONG 0xb782 DEFINED (__AltInterrupt113)?<code 337> (__AltInterrupt113):DEFINED (__Interrupt113)?<code 337> (__Interrupt113):<code 337> (__DefaultInterrupt)
                  0x0001f8          0x4 LONG 0xb782 DEFINED (__AltInterrupt114)?<code 337> (__AltInterrupt114):DEFINED (__Interrupt114)?<code 337> (__Interrupt114):<code 337> (__DefaultInterrupt)
                  0x0001fa          0x4 LONG 0xb782 DEFINED (__AltInterrupt115)?<code 337> (__AltInterrupt115):DEFINED (__Interrupt115)?<code 337> (__Interrupt115):<code 337> (__DefaultInterrupt)
                  0x0001fc          0x4 LONG 0xb782 DEFINED (__AltInterrupt116)?<code 337> (__AltInterrupt116):DEFINED (__Interrupt116)?<code 337> (__Interrupt116):<code 337> (__DefaultInterrupt)
                  0x0001fe          0x4 LONG 0xb782 DEFINED (__AltInterrupt117)?<code 337> (__AltInterrupt117):DEFINED (__Interrupt117)?<code 337> (__Interrupt117):<code 337> (__DefaultInterrupt)
                    0x0000                  WREG0 = 0x0
                    0x0000                  _WREG0 = 0x0
                    0x0002                  WREG1 = 0x2
                    0x0002                  _WREG1 = 0x2
                    0x0004                  WREG2 = 0x4
                    0x0004                  _WREG2 = 0x4
                    0x0006                  WREG3 = 0x6
                    0x0006                  _WREG3 = 0x6
                    0x0008                  WREG4 = 0x8
                    0x0008                  _WREG4 = 0x8
                    0x000a                  WREG5 = 0xa
                    0x000a                  _WREG5 = 0xa
                    0x000c                  WREG6 = 0xc
                    0x000c                  _WREG6 = 0xc
                    0x000e                  WREG7 = 0xe
                    0x000e                  _WREG7 = 0xe
                    0x0010                  WREG8 = 0x10
                    0x0010                  _WREG8 = 0x10
                    0x0012                  WREG9 = 0x12
                    0x0012                  _WREG9 = 0x12
                    0x0014                  WREG10 = 0x14
                    0x0014                  _WREG10 = 0x14
                    0x0016                  WREG11 = 0x16
                    0x0016                  _WREG11 = 0x16
                    0x0018                  WREG12 = 0x18
                    0x0018                  _WREG12 = 0x18
                    0x001a                  WREG13 = 0x1a
                    0x001a                  _WREG13 = 0x1a
                    0x001c                  WREG14 = 0x1c
                    0x001c                  _WREG14 = 0x1c
                    0x001e                  WREG15 = 0x1e
                    0x001e                  _WREG15 = 0x1e
                    0x0020                  SPLIM = 0x20
                    0x0020                  _SPLIM = 0x20
                    0x002e                  PCL = 0x2e
                    0x002e                  _PCL = 0x2e
                    0x0030                  PCH = 0x30
                    0x0030                  _PCH = 0x30
                    0x0032                  TBLPAG = 0x32
                    0x0032                  _TBLPAG = 0x32
                    0x0034                  PSVPAG = 0x34
                    0x0034                  _PSVPAG = 0x34
                    0x0036                  RCOUNT = 0x36
                    0x0036                  _RCOUNT = 0x36
                    0x0042                  SR = 0x42
                    0x0042                  _SR = 0x42
                    0x0042                  _SRbits = 0x42
                    0x0044                  CORCON = 0x44
                    0x0044                  _CORCON = 0x44
                    0x0044                  _CORCONbits = 0x44
                    0x0052                  DISICNT = 0x52
                    0x0052                  _DISICNT = 0x52
                    0x0060                  CNEN1 = 0x60
                    0x0060                  _CNEN1 = 0x60
                    0x0060                  _CNEN1bits = 0x60
                    0x0062                  CNEN2 = 0x62
                    0x0062                  _CNEN2 = 0x62
                    0x0062                  _CNEN2bits = 0x62
                    0x0068                  CNPU1 = 0x68
                    0x0068                  _CNPU1 = 0x68
                    0x0068                  _CNPU1bits = 0x68
                    0x006a                  CNPU2 = 0x6a
                    0x006a                  _CNPU2 = 0x6a
                    0x006a                  _CNPU2bits = 0x6a
                    0x0080                  INTCON1 = 0x80
                    0x0080                  _INTCON1 = 0x80
                    0x0080                  _INTCON1bits = 0x80
                    0x0082                  INTCON2 = 0x82
                    0x0082                  _INTCON2 = 0x82
                    0x0082                  _INTCON2bits = 0x82
                    0x0084                  IFS0 = 0x84
                    0x0084                  _IFS0 = 0x84
                    0x0084                  _IFS0bits = 0x84
                    0x0086                  IFS1 = 0x86
                    0x0086                  _IFS1 = 0x86
                    0x0086                  _IFS1bits = 0x86
                    0x0088                  IFS2 = 0x88
                    0x0088                  _IFS2 = 0x88
                    0x0088                  _IFS2bits = 0x88
                    0x008a                  IFS3 = 0x8a
                    0x008a                  _IFS3 = 0x8a
                    0x008a                  _IFS3bits = 0x8a
                    0x008c                  IFS4 = 0x8c
                    0x008c                  _IFS4 = 0x8c
                    0x008c                  _IFS4bits = 0x8c
                    0x0094                  IEC0 = 0x94
                    0x0094                  _IEC0 = 0x94
                    0x0094                  _IEC0bits = 0x94
                    0x0096                  IEC1 = 0x96
                    0x0096                  _IEC1 = 0x96
                    0x0096                  _IEC1bits = 0x96
                    0x0098                  IEC2 = 0x98
                    0x0098                  _IEC2 = 0x98
                    0x0098                  _IEC2bits = 0x98
                    0x009a                  IEC3 = 0x9a
                    0x009a                  _IEC3 = 0x9a
                    0x009a                  _IEC3bits = 0x9a
                    0x009c                  IEC4 = 0x9c
                    0x009c                  _IEC4 = 0x9c
                    0x009c                  _IEC4bits = 0x9c
                    0x00a4                  IPC0 = 0xa4
                    0x00a4                  _IPC0 = 0xa4
                    0x00a4                  _IPC0bits = 0xa4
                    0x00a6                  IPC1 = 0xa6
                    0x00a6                  _IPC1 = 0xa6
                    0x00a6                  _IPC1bits = 0xa6
                    0x00a8                  IPC2 = 0xa8
                    0x00a8                  _IPC2 = 0xa8
                    0x00a8                  _IPC2bits = 0xa8
                    0x00aa                  IPC3 = 0xaa
                    0x00aa                  _IPC3 = 0xaa
                    0x00aa                  _IPC3bits = 0xaa
                    0x00ac                  IPC4 = 0xac
                    0x00ac                  _IPC4 = 0xac
                    0x00ac                  _IPC4bits = 0xac
                    0x00ae                  IPC5 = 0xae
                    0x00ae                  _IPC5 = 0xae
                    0x00ae                  _IPC5bits = 0xae
                    0x00b0                  IPC6 = 0xb0
                    0x00b0                  _IPC6 = 0xb0
                    0x00b0                  _IPC6bits = 0xb0
                    0x00b2                  IPC7 = 0xb2
                    0x00b2                  _IPC7 = 0xb2
                    0x00b2                  _IPC7bits = 0xb2
                    0x00b4                  IPC8 = 0xb4
                    0x00b4                  _IPC8 = 0xb4
                    0x00b4                  _IPC8bits = 0xb4
                    0x00b6                  IPC9 = 0xb6
                    0x00b6                  _IPC9 = 0xb6
                    0x00b6                  _IPC9bits = 0xb6
                    0x00b8                  IPC10 = 0xb8
                    0x00b8                  _IPC10 = 0xb8
                    0x00b8                  _IPC10bits = 0xb8
                    0x00ba                  IPC11 = 0xba
                    0x00ba                  _IPC11 = 0xba
                    0x00ba                  _IPC11bits = 0xba
                    0x00bc                  IPC12 = 0xbc
                    0x00bc                  _IPC12 = 0xbc
                    0x00bc                  _IPC12bits = 0xbc
                    0x00be                  IPC13 = 0xbe
                    0x00be                  _IPC13 = 0xbe
                    0x00be                  _IPC13bits = 0xbe
                    0x00c2                  IPC15 = 0xc2
                    0x00c2                  _IPC15 = 0xc2
                    0x00c2                  _IPC15bits = 0xc2
                    0x00c4                  IPC16 = 0xc4
                    0x00c4                  _IPC16 = 0xc4
                    0x00c4                  _IPC16bits = 0xc4
                    0x0100                  TMR1 = 0x100
                    0x0100                  _TMR1 = 0x100
                    0x0102                  PR1 = 0x102
                    0x0102                  _PR1 = 0x102
                    0x0104                  T1CON = 0x104
                    0x0104                  _T1CON = 0x104
                    0x0104                  _T1CONbits = 0x104
                    0x0106                  TMR2 = 0x106
                    0x0106                  _TMR2 = 0x106
                    0x0108                  TMR3HLD = 0x108
                    0x0108                  _TMR3HLD = 0x108
                    0x010a                  TMR3 = 0x10a
                    0x010a                  _TMR3 = 0x10a
                    0x010c                  PR2 = 0x10c
                    0x010c                  _PR2 = 0x10c
                    0x010e                  PR3 = 0x10e
                    0x010e                  _PR3 = 0x10e
                    0x0110                  T2CON = 0x110
                    0x0110                  _T2CON = 0x110
                    0x0110                  _T2CONbits = 0x110
                    0x0112                  T3CON = 0x112
                    0x0112                  _T3CON = 0x112
                    0x0112                  _T3CONbits = 0x112
                    0x0114                  TMR4 = 0x114
                    0x0114                  _TMR4 = 0x114
                    0x0116                  TMR5HLD = 0x116
                    0x0116                  _TMR5HLD = 0x116
                    0x0118                  TMR5 = 0x118
                    0x0118                  _TMR5 = 0x118
                    0x011a                  PR4 = 0x11a
                    0x011a                  _PR4 = 0x11a
                    0x011c                  PR5 = 0x11c
                    0x011c                  _PR5 = 0x11c
                    0x011e                  T4CON = 0x11e
                    0x011e                  _T4CON = 0x11e
                    0x011e                  _T4CONbits = 0x11e
                    0x0120                  T5CON = 0x120
                    0x0120                  _T5CON = 0x120
                    0x0120                  _T5CONbits = 0x120
                    0x0140                  IC1BUF = 0x140
                    0x0140                  _IC1BUF = 0x140
                    0x0142                  IC1CON = 0x142
                    0x0142                  _IC1CON = 0x142
                    0x0142                  _IC1CONbits = 0x142
                    0x0144                  IC2BUF = 0x144
                    0x0144                  _IC2BUF = 0x144
                    0x0146                  IC2CON = 0x146
                    0x0146                  _IC2CON = 0x146
                    0x0146                  _IC2CONbits = 0x146
                    0x0148                  IC3BUF = 0x148
                    0x0148                  _IC3BUF = 0x148
                    0x014a                  IC3CON = 0x14a
                    0x014a                  _IC3CON = 0x14a
                    0x014a                  _IC3CONbits = 0x14a
                    0x014c                  IC4BUF = 0x14c
                    0x014c                  _IC4BUF = 0x14c
                    0x014e                  IC4CON = 0x14e
                    0x014e                  _IC4CON = 0x14e
                    0x014e                  _IC4CONbits = 0x14e
                    0x0150                  IC5BUF = 0x150
                    0x0150                  _IC5BUF = 0x150
                    0x0152                  IC5CON = 0x152
                    0x0152                  _IC5CON = 0x152
                    0x0152                  _IC5CONbits = 0x152
                    0x0180                  OC1RS = 0x180
                    0x0180                  _OC1RS = 0x180
                    0x0182                  OC1R = 0x182
                    0x0182                  _OC1R = 0x182
                    0x0184                  OC1CON = 0x184
                    0x0184                  _OC1CON = 0x184
                    0x0184                  _OC1CONbits = 0x184
                    0x0186                  OC2RS = 0x186
                    0x0186                  _OC2RS = 0x186
                    0x0188                  OC2R = 0x188
                    0x0188                  _OC2R = 0x188
                    0x018a                  OC2CON = 0x18a
                    0x018a                  _OC2CON = 0x18a
                    0x018a                  _OC2CONbits = 0x18a
                    0x018c                  OC3RS = 0x18c
                    0x018c                  _OC3RS = 0x18c
                    0x018e                  OC3R = 0x18e
                    0x018e                  _OC3R = 0x18e
                    0x0190                  OC3CON = 0x190
                    0x0190                  _OC3CON = 0x190
                    0x0190                  _OC3CONbits = 0x190
                    0x0192                  OC4RS = 0x192
                    0x0192                  _OC4RS = 0x192
                    0x0194                  OC4R = 0x194
                    0x0194                  _OC4R = 0x194
                    0x0196                  OC4CON = 0x196
                    0x0196                  _OC4CON = 0x196
                    0x0196                  _OC4CONbits = 0x196
                    0x0198                  OC5RS = 0x198
                    0x0198                  _OC5RS = 0x198
                    0x019a                  OC5R = 0x19a
                    0x019a                  _OC5R = 0x19a
                    0x019c                  OC5CON = 0x19c
                    0x019c                  _OC5CON = 0x19c
                    0x019c                  _OC5CONbits = 0x19c
                    0x0200                  I2C1RCV = 0x200
                    0x0200                  _I2C1RCV = 0x200
                    0x0202                  I2C1TRN = 0x202
                    0x0202                  _I2C1TRN = 0x202
                    0x0204                  I2C1BRG = 0x204
                    0x0204                  _I2C1BRG = 0x204
                    0x0206                  I2C1CON = 0x206
                    0x0206                  _I2C1CON = 0x206
                    0x0206                  _I2C1CONbits = 0x206
                    0x0208                  I2C1STAT = 0x208
                    0x0208                  _I2C1STAT = 0x208
                    0x0208                  _I2C1STATbits = 0x208
                    0x020a                  I2C1ADD = 0x20a
                    0x020a                  _I2C1ADD = 0x20a
                    0x020c                  I2C1MSK = 0x20c
                    0x020c                  _I2C1MSK = 0x20c
                    0x0210                  I2C2RCV = 0x210
                    0x0210                  _I2C2RCV = 0x210
                    0x0212                  I2C2TRN = 0x212
                    0x0212                  _I2C2TRN = 0x212
                    0x0214                  I2C2BRG = 0x214
                    0x0214                  _I2C2BRG = 0x214
                    0x0216                  I2C2CON = 0x216
                    0x0216                  _I2C2CON = 0x216
                    0x0216                  _I2C2CONbits = 0x216
                    0x0218                  I2C2STAT = 0x218
                    0x0218                  _I2C2STAT = 0x218
                    0x0218                  _I2C2STATbits = 0x218
                    0x021a                  I2C2ADD = 0x21a
                    0x021a                  _I2C2ADD = 0x21a
                    0x021c                  I2C2MSK = 0x21c
                    0x021c                  _I2C2MSK = 0x21c
                    0x0220                  U1MODE = 0x220
                    0x0220                  _U1MODE = 0x220
                    0x0220                  _U1MODEbits = 0x220
                    0x0222                  U1STA = 0x222
                    0x0222                  _U1STA = 0x222
                    0x0222                  _U1STAbits = 0x222
                    0x0224                  U1TXREG = 0x224
                    0x0224                  _U1TXREG = 0x224
                    0x0226                  U1RXREG = 0x226
                    0x0226                  _U1RXREG = 0x226
                    0x0228                  U1BRG = 0x228
                    0x0228                  _U1BRG = 0x228
                    0x0230                  U2MODE = 0x230
                    0x0230                  _U2MODE = 0x230
                    0x0230                  _U2MODEbits = 0x230
                    0x0232                  U2STA = 0x232
                    0x0232                  _U2STA = 0x232
                    0x0232                  _U2STAbits = 0x232
                    0x0234                  U2TXREG = 0x234
                    0x0234                  _U2TXREG = 0x234
                    0x0236                  U2RXREG = 0x236
                    0x0236                  _U2RXREG = 0x236
                    0x0238                  U2BRG = 0x238
                    0x0238                  _U2BRG = 0x238
                    0x0240                  SPI1STAT = 0x240
                    0x0240                  _SPI1STAT = 0x240
                    0x0240                  _SPI1STATbits = 0x240
                    0x0242                  SPI1CON1 = 0x242
                    0x0242                  _SPI1CON1 = 0x242
                    0x0242                  _SPI1CON1bits = 0x242
                    0x0244                  SPI1CON2 = 0x244
                    0x0244                  _SPI1CON2 = 0x244
                    0x0244                  _SPI1CON2bits = 0x244
                    0x0248                  SPI1BUF = 0x248
                    0x0248                  _SPI1BUF = 0x248
                    0x0260                  SPI2STAT = 0x260
                    0x0260                  _SPI2STAT = 0x260
                    0x0260                  _SPI2STATbits = 0x260
                    0x0262                  SPI2CON1 = 0x262
                    0x0262                  _SPI2CON1 = 0x262
                    0x0262                  _SPI2CON1bits = 0x262
                    0x0264                  SPI2CON2 = 0x264
                    0x0264                  _SPI2CON2 = 0x264
                    0x0264                  _SPI2CON2bits = 0x264
                    0x0268                  SPI2BUF = 0x268
                    0x0268                  _SPI2BUF = 0x268
                    0x02c0                  TRISA = 0x2c0
                    0x02c0                  _TRISA = 0x2c0
                    0x02c0                  _TRISAbits = 0x2c0
                    0x02c2                  PORTA = 0x2c2
                    0x02c2                  _PORTA = 0x2c2
                    0x02c2                  _PORTAbits = 0x2c2
                    0x02c4                  LATA = 0x2c4
                    0x02c4                  _LATA = 0x2c4
                    0x02c4                  _LATAbits = 0x2c4
                    0x02c6                  TRISB = 0x2c6
                    0x02c6                  _TRISB = 0x2c6
                    0x02c6                  _TRISBbits = 0x2c6
                    0x02c8                  PORTB = 0x2c8
                    0x02c8                  _PORTB = 0x2c8
                    0x02c8                  _PORTBbits = 0x2c8
                    0x02ca                  LATB = 0x2ca
                    0x02ca                  _LATB = 0x2ca
                    0x02ca                  _LATBbits = 0x2ca
                    0x02cc                  TRISC = 0x2cc
                    0x02cc                  _TRISC = 0x2cc
                    0x02cc                  _TRISCbits = 0x2cc
                    0x02ce                  PORTC = 0x2ce
                    0x02ce                  _PORTC = 0x2ce
                    0x02ce                  _PORTCbits = 0x2ce
                    0x02d0                  LATC = 0x2d0
                    0x02d0                  _LATC = 0x2d0
                    0x02d0                  _LATCbits = 0x2d0
                    0x02d2                  TRISD = 0x2d2
                    0x02d2                  _TRISD = 0x2d2
                    0x02d2                  _TRISDbits = 0x2d2
                    0x02d4                  PORTD = 0x2d4
                    0x02d4                  _PORTD = 0x2d4
                    0x02d4                  _PORTDbits = 0x2d4
                    0x02d6                  LATD = 0x2d6
                    0x02d6                  _LATD = 0x2d6
                    0x02d6                  _LATDbits = 0x2d6
                    0x02d8                  TRISE = 0x2d8
                    0x02d8                  _TRISE = 0x2d8
                    0x02d8                  _TRISEbits = 0x2d8
                    0x02da                  PORTE = 0x2da
                    0x02da                  _PORTE = 0x2da
                    0x02da                  _PORTEbits = 0x2da
                    0x02dc                  LATE = 0x2dc
                    0x02dc                  _LATE = 0x2dc
                    0x02dc                  _LATEbits = 0x2dc
                    0x02de                  TRISF = 0x2de
                    0x02de                  _TRISF = 0x2de
                    0x02de                  _TRISFbits = 0x2de
                    0x02e0                  PORTF = 0x2e0
                    0x02e0                  _PORTF = 0x2e0
                    0x02e0                  _PORTFbits = 0x2e0
                    0x02e2                  LATF = 0x2e2
                    0x02e2                  _LATF = 0x2e2
                    0x02e2                  _LATFbits = 0x2e2
                    0x02e4                  TRISG = 0x2e4
                    0x02e4                  _TRISG = 0x2e4
                    0x02e4                  _TRISGbits = 0x2e4
                    0x02e6                  PORTG = 0x2e6
                    0x02e6                  _PORTG = 0x2e6
                    0x02e6                  _PORTGbits = 0x2e6
                    0x02e8                  LATG = 0x2e8
                    0x02e8                  _LATG = 0x2e8
                    0x02e8                  _LATGbits = 0x2e8
                    0x02fc                  PADCFG1 = 0x2fc
                    0x02fc                  _PADCFG1 = 0x2fc
                    0x02fc                  _PADCFG1bits = 0x2fc
                    0x0300                  ADC1BUF0 = 0x300
                    0x0300                  _ADC1BUF0 = 0x300
                    0x0302                  ADC1BUF1 = 0x302
                    0x0302                  _ADC1BUF1 = 0x302
                    0x0304                  ADC1BUF2 = 0x304
                    0x0304                  _ADC1BUF2 = 0x304
                    0x0306                  ADC1BUF3 = 0x306
                    0x0306                  _ADC1BUF3 = 0x306
                    0x0308                  ADC1BUF4 = 0x308
                    0x0308                  _ADC1BUF4 = 0x308
                    0x030a                  ADC1BUF5 = 0x30a
                    0x030a                  _ADC1BUF5 = 0x30a
                    0x030c                  ADC1BUF6 = 0x30c
                    0x030c                  _ADC1BUF6 = 0x30c
                    0x030e                  ADC1BUF7 = 0x30e
                    0x030e                  _ADC1BUF7 = 0x30e
                    0x0310                  ADC1BUF8 = 0x310
                    0x0310                  _ADC1BUF8 = 0x310
                    0x0312                  ADC1BUF9 = 0x312
                    0x0312                  _ADC1BUF9 = 0x312
                    0x0314                  ADC1BUFA = 0x314
                    0x0314                  _ADC1BUFA = 0x314
                    0x0316                  ADC1BUFB = 0x316
                    0x0316                  _ADC1BUFB = 0x316
                    0x0318                  ADC1BUFC = 0x318
                    0x0318                  _ADC1BUFC = 0x318
                    0x031a                  ADC1BUFD = 0x31a
                    0x031a                  _ADC1BUFD = 0x31a
                    0x031c                  ADC1BUFE = 0x31c
                    0x031c                  _ADC1BUFE = 0x31c
                    0x031e                  ADC1BUFF = 0x31e
                    0x031e                  _ADC1BUFF = 0x31e
                    0x0320                  AD1CON1 = 0x320
                    0x0320                  _AD1CON1 = 0x320
                    0x0320                  _AD1CON1bits = 0x320
                    0x0322                  AD1CON2 = 0x322
                    0x0322                  _AD1CON2 = 0x322
                    0x0322                  _AD1CON2bits = 0x322
                    0x0324                  AD1CON3 = 0x324
                    0x0324                  _AD1CON3 = 0x324
                    0x0324                  _AD1CON3bits = 0x324
                    0x0328                  AD1CHS = 0x328
                    0x0328                  _AD1CHS = 0x328
                    0x0328                  _AD1CHSbits = 0x328
                    0x032c                  AD1PCFG = 0x32c
                    0x032c                  _AD1PCFG = 0x32c
                    0x032c                  _AD1PCFGbits = 0x32c
                    0x0330                  AD1CSSL = 0x330
                    0x0330                  _AD1CSSL = 0x330
                    0x0330                  _AD1CSSLbits = 0x330
                    0x0600                  PMCON = 0x600
                    0x0600                  _PMCON = 0x600
                    0x0600                  _PMCONbits = 0x600
                    0x0602                  PMMODE = 0x602
                    0x0602                  _PMMODE = 0x602
                    0x0602                  _PMMODEbits = 0x602
                    0x0604                  PMADDR = 0x604
                    0x0604                  _PMADDR = 0x604
                    0x0604                  _PMADDRbits = 0x604
                    0x0604                  PMDOUT1 = 0x604
                    0x0604                  _PMDOUT1 = 0x604
                    0x0604                  _PMDOUT1bits = 0x604
                    0x0606                  PMDOUT2 = 0x606
                    0x0606                  _PMDOUT2 = 0x606
                    0x0608                  PMDIN1 = 0x608
                    0x0608                  _PMDIN1 = 0x608
                    0x060a                  PMDIN2 = 0x60a
                    0x060a                  _PMDIN2 = 0x60a
                    0x060c                  PMAEN = 0x60c
                    0x060c                  _PMAEN = 0x60c
                    0x060c                  _PMAENbits = 0x60c
                    0x060e                  PMSTAT = 0x60e
                    0x060e                  _PMSTAT = 0x60e
                    0x060e                  _PMSTATbits = 0x60e
                    0x0620                  ALRMVAL = 0x620
                    0x0620                  _ALRMVAL = 0x620
                    0x0622                  ALCFGRPT = 0x622
                    0x0622                  _ALCFGRPT = 0x622
                    0x0622                  _ALCFGRPTbits = 0x622
                    0x0624                  RTCVAL = 0x624
                    0x0624                  _RTCVAL = 0x624
                    0x0626                  RCFGCAL = 0x626
                    0x0626                  _RCFGCAL = 0x626
                    0x0626                  _RCFGCALbits = 0x626
                    0x0630                  CMCON = 0x630
                    0x0630                  _CMCON = 0x630
                    0x0630                  _CMCONbits = 0x630
                    0x0632                  CVRCON = 0x632
                    0x0632                  _CVRCON = 0x632
                    0x0632                  _CVRCONbits = 0x632
                    0x0640                  CRCCON = 0x640
                    0x0640                  _CRCCON = 0x640
                    0x0640                  _CRCCONbits = 0x640
                    0x0642                  CRCXOR = 0x642
                    0x0642                  _CRCXOR = 0x642
                    0x0642                  _CRCXORbits = 0x642
                    0x0644                  CRCDAT = 0x644
                    0x0644                  _CRCDAT = 0x644
                    0x0646                  CRCWDAT = 0x646
                    0x0646                  _CRCWDAT = 0x646
                    0x06c0                  ODCA = 0x6c0
                    0x06c0                  _ODCA = 0x6c0
                    0x06c0                  _ODCAbits = 0x6c0
                    0x06c6                  ODCB = 0x6c6
                    0x06c6                  _ODCB = 0x6c6
                    0x06c6                  _ODCBbits = 0x6c6
                    0x06cc                  ODCC = 0x6cc
                    0x06cc                  _ODCC = 0x6cc
                    0x06cc                  _ODCCbits = 0x6cc
                    0x06d2                  ODCD = 0x6d2
                    0x06d2                  _ODCD = 0x6d2
                    0x06d2                  _ODCDbits = 0x6d2
                    0x06d8                  ODCE = 0x6d8
                    0x06d8                  _ODCE = 0x6d8
                    0x06d8                  _ODCEbits = 0x6d8
                    0x06de                  ODCF = 0x6de
                    0x06de                  _ODCF = 0x6de
                    0x06de                  _ODCFbits = 0x6de
                    0x06e4                  ODCG = 0x6e4
                    0x06e4                  _ODCG = 0x6e4
                    0x06e4                  _ODCGbits = 0x6e4
                    0x0740                  RCON = 0x740
                    0x0740                  _RCON = 0x740
                    0x0740                  _RCONbits = 0x740
                    0x0742                  OSCCON = 0x742
                    0x0742                  _OSCCON = 0x742
                    0x0742                  _OSCCONbits = 0x742
                    0x0742                  OSCCONL = 0x742
                    0x0742                  _OSCCONL = 0x742
                    0x0743                  OSCCONH = 0x743
                    0x0743                  _OSCCONH = 0x743
                    0x0744                  CLKDIV = 0x744
                    0x0744                  _CLKDIV = 0x744
                    0x0744                  _CLKDIVbits = 0x744
                    0x0748                  OSCTUN = 0x748
                    0x0748                  _OSCTUN = 0x748
                    0x0748                  _OSCTUNbits = 0x748
                    0x0760                  NVMCON = 0x760
                    0x0760                  _NVMCON = 0x760
                    0x0760                  _NVMCONbits = 0x760
                    0x0766                  NVMKEY = 0x766
                    0x0766                  _NVMKEY = 0x766
                    0x0770                  PMD1 = 0x770
                    0x0770                  _PMD1 = 0x770
                    0x0770                  _PMD1bits = 0x770
                    0x0772                  PMD2 = 0x772
                    0x0772                  _PMD2 = 0x772
                    0x0772                  _PMD2bits = 0x772
                    0x0774                  PMD3 = 0x774
                    0x0774                  _PMD3 = 0x774
                    0x0774                  _PMD3bits = 0x774
                    0x0140                  IC1 = 0x140
                    0x0140                  _IC1 = 0x140
                    0x0144                  IC2 = 0x144
                    0x0144                  _IC2 = 0x144
                    0x0148                  IC3 = 0x148
                    0x0148                  _IC3 = 0x148
                    0x014c                  IC4 = 0x14c
                    0x014c                  _IC4 = 0x14c
                    0x0150                  IC5 = 0x150
                    0x0150                  _IC5 = 0x150
                    0x0180                  OC1 = 0x180
                    0x0180                  _OC1 = 0x180
                    0x0186                  OC2 = 0x186
                    0x0186                  _OC2 = 0x186
                    0x018c                  OC3 = 0x18c
                    0x018c                  _OC3 = 0x18c
                    0x0192                  OC4 = 0x192
                    0x0192                  _OC4 = 0x192
                    0x0198                  OC5 = 0x198
                    0x0198                  _OC5 = 0x198
                    0x0240                  SPI1 = 0x240
                    0x0240                  _SPI1 = 0x240
                    0x0260                  SPI2 = 0x260
                    0x0260                  _SPI2 = 0x260
                    0x0220                  UART1 = 0x220
                    0x0220                  _UART1 = 0x220
                    0x0230                  UART2 = 0x230
                    0x0230                  _UART2 = 0x230
                    0x0001                  __MPLAB_BUILD = 0x1
                    0x0001                  __MPLAB_DEBUG = 0x1
                    0x0001                  __MPLAB_DEBUGGER_REAL_ICE = 0x1
                    0x0001                  __ICD2RAM = 0x1
START GROUP
LOAD c:/program files/microchip/mplab c30/bin/bin/../../lib\libpic30-coff.a
LOAD c:/program files/microchip/mplab c30/bin/bin/../../lib\libm-coff.a
LOAD c:/program files/microchip/mplab c30/bin/bin/../../lib\libc-coff.a
END GROUP
OUTPUT(TCPIP Demo App-C30.cof coff-pic30)
LOAD data_init
LOAD default_isr

.nbss               0x0850        0x38e
 .nbss              0x0850        0x19a ..\Microchip\TCPIP Stack\Objects - TCPIP Demo App-C30\TCP.o
 .nbss              0x09ea         0x98 ..\Microchip\TCPIP Stack\Objects - TCPIP Demo App-C30\UDP.o
                    0x09f0                  UDPSocketInfo
                    0x0a7c                  activeUDPSocket
                    0x0a7e                  UDPTxCount
                    0x0a80                  UDPRxCount
 .nbss              0x0a82         0x8c ..\Microchip\TCPIP Stack\Objects - TCPIP Demo App-C30\HTTP2.o
                    0x0a82                  curHTTP
                    0x0b04                  httpStubs
                    0x0b0c                  curHTTPID
 .nbss              0x0b0e         0x6c ..\Microchip\TCPIP Stack\Objects - TCPIP Demo App-C30\MPFS2.o
 .nbss              0x0b7a         0x64 Objects - TCPIP Demo App-C30\CustomHTTPApp.o
                    0x0b7a                  bufName
                    0x0bac                  bufFact

.ndata              0x0bde         0x90
 .ndata             0x0bde         0x48 ..\Microchip\TCPIP Stack\Objects - TCPIP Demo App-C30\HTTP2.o
 .ndata             0x0c26         0x48 Objects - TCPIP Demo App-C30\SMTPDemo.o

.nbss               0x0c6e        0x116
 .nbss              0x0c6e         0x40 Objects - TCPIP Demo App-C30\MainDemo.o
                    0x0c72                  AppConfig
                    0x0ca5                  AN0String
 .nbss              0x0cae         0x40 ..\Microchip\TCPIP Stack\Objects - TCPIP Demo App-C30\Hashes.o
                    0x0cae                  lastBlock
 .nbss              0x0cee         0x3a ..\Microchip\TCPIP Stack\Objects - TCPIP Demo App-C30\DynDNS.o
                    0x0d18                  DDNSClient
 .nbss              0x0d28         0x3a ..\Microchip\TCPIP Stack\Objects - TCPIP Demo App-C30\SMTP.o
                    0x0d4a                  SMTPClient
 .nbss              0x0d62         0x22 ..\Microchip\TCPIP Stack\Objects - TCPIP Demo App-C30\DHCP.o

.ndata              0x0d84         0x22
 .ndata             0x0d84         0x22 ..\Microchip\TCPIP Stack\Objects - TCPIP Demo App-C30\DynDNS.o
                    0x0d9e                  ddnsServiceHosts

.nbss               0x0da6         0x76
 .nbss              0x0da6         0x22 ..\Microchip\TCPIP Stack\Objects - TCPIP Demo App-C30\LCDBlocking.o
                    0x0da6                  LCDText
 .nbss              0x0dc8         0x18 ..\Microchip\TCPIP Stack\Objects - TCPIP Demo App-C30\DNS.o
 .nbss              0x0de0         0x16 ..\Microchip\TCPIP Stack\Objects - TCPIP Demo App-C30\ARP.o
 .nbss              0x0df6          0xc ..\Microchip\TCPIP Stack\Objects - TCPIP Demo App-C30\StackTsk.o
                    0x0df8                  remoteNode
 .nbss              0x0e02          0xa ..\Microchip\TCPIP Stack\Objects - TCPIP Demo App-C30\Tick.o
 .nbss              0x0e0c          0x8 ..\Microchip\TCPIP Stack\Objects - TCPIP Demo App-C30\DHCPs.o
 .nbss              0x0e14          0x8 ..\Microchip\TCPIP Stack\Objects - TCPIP Demo App-C30\ENC28J60.o

.ndata              0x0e1c          0x6
 .ndata             0x0e1c          0x6 ..\Microchip\TCPIP Stack\Objects - TCPIP Demo App-C30\DHCP.o
                    0x0e1c                  smDHCPState
                    0x0e1e                  DHCPFlags
                    0x0e20                  DHCPBindCount

.nbss               0x0e22          0x6
 .nbss              0x0e22          0x6 Objects - TCPIP Demo App-C30\SMTPDemo.o

.ndata              0x0e28          0x8
 .ndata             0x0e28          0x4 Objects - TCPIP Demo App-C30\MainDemo.o
                    0x0e28                  myDHCPBindCount
                    0x0e2a                  __C30_UART
 .ndata             0x0e2c          0x4 ..\Microchip\TCPIP Stack\Objects - TCPIP Demo App-C30\DNS.o

.nbss               0x0e30          0x8
 .nbss              0x0e30          0x4 ..\Microchip\TCPIP Stack\Objects - TCPIP Demo App-C30\IP.o
 .nbss              0x0e34          0x4 ..\Microchip\TCPIP Stack\Objects - TCPIP Demo App-C30\NBNS.o

.ndata              0x0e38          0x2
 .ndata             0x0e38          0x2 ..\Microchip\TCPIP Stack\Objects - TCPIP Demo App-C30\UDP.o

_014c8af04a4a21c5
                    0x0e3a          0x2
 _014c8af04a4a21c5
                    0x0e3a          0x2 ..\Microchip\TCPIP Stack\Objects - TCPIP Demo App-C30\UDP.o

.ndata              0x0e3c          0x2
 .ndata             0x0e3c          0x2 ..\Microchip\TCPIP Stack\Objects - TCPIP Demo App-C30\DHCPs.o
                    0x0e3c                  bDHCPServerEnabled

_014bfc404a4a21cb
                    0x0e3e          0x2
 _014bfc404a4a21cb
                    0x0e3e          0x2 ..\Microchip\TCPIP Stack\Objects - TCPIP Demo App-C30\DNS.o

.ndata              0x0e40          0x4
 .ndata             0x0e40          0x2 ..\Microchip\TCPIP Stack\Objects - TCPIP Demo App-C30\SMTP.o
 .ndata             0x0e42          0x2 ..\Microchip\TCPIP Stack\Objects - TCPIP Demo App-C30\TCP.o

_014d9b604a4a21dc
                    0x0e44          0x2
 _014d9b604a4a21dc
                    0x0e44          0x2 ..\Microchip\TCPIP Stack\Objects - TCPIP Demo App-C30\TCP.o

.bss                0x0e46         0x88
 .bss               0x0e46         0x88 c:/program files/microchip/mplab c30/bin/bin/../../lib\libc-coff.a(rand.o)

.data               0x0ece         0x58
 .data              0x0ece         0x4a c:/program files/microchip/mplab c30/bin/bin/../../lib\libc-coff.a(xstoul.o)
 .data              0x0f18          0xa c:/program files/microchip/mplab c30/bin/bin/../../lib\libc-coff.a(rand.o)
                    0x0f18                  _Tls_setup__Randseed
                    0x0f1a                  _Randseed
                    0x0f1e                  _Tls_setup__Randinit
                    0x0f20                  _Randinit
 .data              0x0f22          0x4 c:/program files/microchip/mplab c30/bin/bin/../../lib\libc-coff.a(errno.o)
                    0x0f22                  _Tls_setup_errno
                    0x0f24                  errno

.const              0x87a0        0x88e load address 0x0007a0  
 .const             0x87a0        0x3fe ..\Microchip\TCPIP Stack\Objects - TCPIP Demo App-C30\HTTP2.o
 .const             0x8b9e        0x1a4 ..\Microchip\TCPIP Stack\Objects - TCPIP Demo App-C30\DynDNS.o
 .const             0x8d42        0x140 ..\Microchip\TCPIP Stack\Objects - TCPIP Demo App-C30\Hashes.o
 .const             0x8e82         0x86 ..\Microchip\TCPIP Stack\Objects - TCPIP Demo App-C30\SMTP.o
 .const             0x8f08         0x68 Objects - TCPIP Demo App-C30\CustomHTTPApp.o
 .const             0x8f70         0x4a Objects - TCPIP Demo App-C30\SMTPDemo.o
 .const             0x8fba         0x36 ..\Microchip\TCPIP Stack\Objects - TCPIP Demo App-C30\TCP.o
                    0x8fba                  TCPSocketInitializer
 .const             0x8ff0         0x32 Objects - TCPIP Demo App-C30\MainDemo.o
 .const             0x9022          0x8 ..\Microchip\TCPIP Stack\Objects - TCPIP Demo App-C30\MPFS2.o
 .const             0x902a          0x4 Objects - TCPIP Demo App-C30\MPFSImg2-C30.o
                    0x902a                  MPFS_Start

.text             0x00102e       0x20c8
 .text            0x00102e       0x20c8 ..\Microchip\TCPIP Stack\Objects - TCPIP Demo App-C30\TCP.o
                  0x0010ca                  TCPInit
                  0x001190                  TCPOpen
                  0x0012d6                  TCPWasReset
                  0x0012fa                  TCPIsConnected
                  0x001316                  TCPDisconnect
                  0x001398                  TCPGetRemoteInfo
                  0x0013b4                  TCPFlush
                  0x0013d0                  TCPIsPutReady
                  0x00141a                  TCPPut
                  0x0014a6                  TCPPutArray
                  0x001574                  TCPPutString
                  0x001592                  TCPGetTxFIFOFull
                  0x0015b0                  TCPDiscard
                  0x0015ce                  TCPIsGetReady
                  0x001600                  TCPGet
                  0x00166a                  TCPGetArray
                  0x001726                  TCPGetRxFIFOFree
                  0x001742                  TCPFindArrayEx
                  0x0019c6                  TCPFindEx
                  0x0019e4                  TCPTick
                  0x001e52                  TCPProcess
                  0x002edc                  TCPAdjustFIFOSize

.text             0x0030f6       0x152a
 .text            0x0030f6       0x152a ..\Microchip\TCPIP Stack\Objects - TCPIP Demo App-C30\HTTP2.o
                  0x0030f6                  HTTPPrint
                  0x003116                  HTTPPrint_
                  0x003130                  HTTPInit
                  0x0031a0                  HTTPServer
                  0x004246                  HTTPURLDecode
                  0x00430c                  HTTPGetArg
                  0x004354                  HTTPReadPostName
                  0x00437c                  HTTPReadPostValue
                  0x004558                  HTTPIncFile

.text             0x004620        0xec0
 .text            0x004620        0xec0 ..\Microchip\TCPIP Stack\Objects - TCPIP Demo App-C30\SMTP.o
                  0x004620                  SMTPBeginUsage
                  0x004674                  SMTPEndUsage
                  0x0046bc                  SMTPTask
                  0x005218                  SMTPSendMail
                  0x005220                  SMTPIsBusy
                  0x005236                  SMTPIsPutReady
                  0x005252                  SMTPPut
                  0x0052f2                  SMTPPutArray
                  0x00532e                  SMTPPutString
                  0x005364                  SMTPFlush
                  0x005370                  SMTPPutDone

.text             0x0054e0        0xcb6
 .text            0x0054e0        0xcb6 ..\Microchip\TCPIP Stack\Objects - TCPIP Demo App-C30\ENC28J60.o
                  0x0054e0                  MACInit
                  0x005600                  MACIsLinked
                  0x005614                  MACIsTxReady
                  0x00562c                  MACDiscardRx
                  0x005660                  MACGetFreeRxSize
                  0x0056e8                  MACGetHeader
                  0x0057ca                  MACPutHeader
                  0x00581e                  MACFlush
                  0x00593a                  MACSetReadPtrInRx
                  0x005968                  MACSetWritePtr
                  0x005996                  MACSetReadPtr
                  0x0059c4                  MACCalcRxChecksum
                  0x005a1c                  CalcIPBufferChecksum
                  0x005ad0                  MACMemCopyAsync
                  0x005c7e                  MACIsMemCopyDone
                  0x005c96                  MACGet
                  0x005cc8                  MACGetArray
                  0x005da2                  MACPut
                  0x005dda                  MACPutArray
                  0x005f96                  ReadPHYReg
                  0x0060c8                  WritePHYReg
                  0x006118                  MACPowerDown
                  0x006146                  MACPowerUp
                  0x006166                  SetCLKOUT
                  0x00617c                  GetCLKOUT

.text             0x006196        0xb5a
 .text            0x006196        0xb5a ..\Microchip\TCPIP Stack\Objects - TCPIP Demo App-C30\MPFS2.o
                  0x006196                  MPFSInit
                  0x0061c0                  MPFSOpen
                  0x00630e                  MPFSOpenID
                  0x006392                  MPFSClose
                  0x0063b4                  MPFSGet
                  0x00655a                  MPFSGetArray
                  0x0067be                  MPFSGetLong
                  0x0067de                  MPFSSeek
                  0x0069f8                  MPFSGetTimestamp
                  0x006a46                  MPFSGetMicrotime
                  0x006a94                  MPFSGetFlags
                  0x006ad8                  MPFSGetSize
                  0x006b26                  MPFSGetBytesRem
                  0x006b6e                  MPFSGetStartAddr
                  0x006bbe                  MPFSGetEndAddr
                  0x006c18                  MPFSGetFilename
                  0x006c80                  MPFSGetPosition
                  0x006ca0                  MPFSGetID

.text             0x006cf0        0x964
 .text            0x006cf0        0x964 ..\Microchip\TCPIP Stack\Objects - TCPIP Demo App-C30\DynDNS.o
                  0x006cf0                  DDNSInit
                  0x006d32                  DDNSTask
                  0x00760a                  DDNSForceUpdate
                  0x007620                  DDNSSetService
                  0x007640                  DDNSGetLastIP
                  0x00764c                  DDNSGetLastStatus

.text             0x007654        0x956
 .text            0x007654        0x956 ..\Microchip\TCPIP Stack\Objects - TCPIP Demo App-C30\Helpers.o
                  0x007654                  GenerateRandomDWORD
                  0x00776e                  StringToIPAddress
                  0x0078ee                  Base64Decode
                  0x007a54                  Base64Encode
                  0x007bb0                  uitoa
                  0x007c2e                  ultoa
                  0x007cde                  hexatob
                  0x007d54                  btohexa_high
                  0x007d7c                  btohexa_low
                  0x007da2                  stricmppgm2ram
                  0x007e3a                  swaps
                  0x007e54                  swapl
                  0x007eb2                  CalcIPChecksum
                  0x007f28                  strupr
                  0x007f62                  FormatNetBIOSName

.text             0x007faa        0x8d2
 .text            0x007faa        0x8d2 ..\Microchip\TCPIP Stack\Objects - TCPIP Demo App-C30\DHCP.o
                  0x007faa                  DHCPReset
                  0x007fcc                  DHCPDisable
                  0x007fe8                  DHCPEnable
                  0x008000                  DHCPTask

.text             0x00887c        0x792
 .text            0x00887c        0x792 ..\Microchip\TCPIP Stack\Objects - TCPIP Demo App-C30\DNS.o
                  0x00887c                  DNSBeginUsage
                  0x008898                  DNSEndUsage
                  0x0088be                  DNSResolve
                  0x0088ee                  DNSIsResolved

.text             0x00900e        0x532
 .text            0x00900e        0x532 ..\Microchip\TCPIP Stack\Objects - TCPIP Demo App-C30\UDP.o
                  0x00900e                  UDPInit
                  0x009028                  UDPTask
                  0x009032                  UDPOpen
                  0x0090c0                  UDPClose
                  0x0090ea                  UDPSetTxBuffer
                  0x0090fe                  UDPSetRxBuffer
                  0x009112                  UDPIsPutReady
                  0x009148                  UDPPut
                  0x00917c                  UDPPutArray
                  0x0091b4                  UDPPutString
                  0x0091ca                  UDPFlush
                  0x0092a0                  UDPIsGetReady
                  0x0092d0                  UDPGet
                  0x009306                  UDPGetArray
                  0x009350                  UDPDiscard
                  0x00936c                  UDPProcess

.text             0x009540        0x51a
 .text            0x009540        0x51a ..\Microchip\TCPIP Stack\Objects - TCPIP Demo App-C30\DHCPs.o
                  0x009540                  DHCPServerTask

.text             0x009a5a        0x4c4
 .text            0x009a5a        0x4c4 ..\Microchip\TCPIP Stack\Objects - TCPIP Demo App-C30\Hashes.o
                  0x009a5a                  HashAddData
                  0x009a76                  MD5Initialize
                  0x009ab2                  MD5AddData
                  0x009db2                  MD5Calculate

.text             0x009f1e        0x3a8
 .text            0x009f1e        0x3a8 ..\Microchip\TCPIP Stack\Objects - TCPIP Demo App-C30\ARP.o
                  0x009f98                  ARPInit
                  0x009fce                  ARPProcess
                  0x00a0ce                  ARPResolve
                  0x00a19a                  ARPIsResolved

.text             0x00a2c6        0x386
 .text            0x00a2c6        0x386 ..\Microchip\TCPIP Stack\Objects - TCPIP Demo App-C30\NBNS.o
                  0x00a2c6                  NBNSTask

.text             0x00a64c        0x31e
 .text            0x00a64c        0x31e Objects - TCPIP Demo App-C30\CustomHTTPApp.o
                  0x00a64c                  HTTPNeedsAuth
                  0x00a682                  HTTPCheckAuth
                  0x00a6b0                  HTTPExecuteGet
                  0x00a8da                  HTTPExecutePost

.text             0x00a96a        0x2e2
 .text            0x00a96a        0x2e2 Objects - TCPIP Demo App-C30\MainDemo.o
                  0x00a96a                  _AddressError
                  0x00a974                  _StackError
                  0x00a97e                  main
                  0x00aa22                  DisplayIPValue

.text             0x00ac4c        0x258
 .text            0x00ac4c        0x258 ..\Microchip\TCPIP Stack\Objects - TCPIP Demo App-C30\StackTsk.o
                  0x00ac4c                  StackInit
                  0x00ac84                  StackTask
                  0x00ae8a                  StackApplications

.text             0x00aea4        0x1ac
 .text            0x00aea4        0x1ac ..\Microchip\TCPIP Stack\Objects - TCPIP Demo App-C30\IP.o
                  0x00aea4                  IPGetHeader
                  0x00af6e                  IPPutHeader
                  0x00b00c                  IPSetRxBuffer

.text             0x00b050        0x1a8
 .text            0x00b050        0x1a8 ..\Microchip\TCPIP Stack\Objects - TCPIP Demo App-C30\LCDBlocking.o
                  0x00b094                  LCDInit
                  0x00b120                  LCDUpdate
                  0x00b1dc                  LCDErase

.dinit            0x00b1f8        0x198
 .dinit           0x00b1f8        0x198 data_init

MPFSData          0x00b390        0x110
 MPFSData         0x00b390        0x110 Objects - TCPIP Demo App-C30\MPFSImg2-C30.o
                  0x00b394                  BEGIN_MPFS

.text             0x00b4a0        0x106
 .text            0x00b4a0        0x106 Objects - TCPIP Demo App-C30\SMTPDemo.o
                  0x00b4a0                  SMTPDemo

.text             0x00b5a6         0xfa
 .text            0x00b5a6         0xfa ..\Microchip\TCPIP Stack\Objects - TCPIP Demo App-C30\Tick.o
                  0x00b5a6                  TickInit
                  0x00b622                  TickGet
                  0x00b62e                  TickGetDiv256
                  0x00b648                  TickGetDiv64K
                  0x00b662                  TickConvertToMilliseconds
                  0x00b688                  _T1Interrupt

.text             0x00b6a0         0x7e
 .text            0x00b6a0         0x7e ..\Microchip\TCPIP Stack\Objects - TCPIP Demo App-C30\ICMP.o
                  0x00b6a0                  ICMPProcess

.text             0x00b71e         0x56
 .text            0x00b71e         0x56 ..\Microchip\TCPIP Stack\Objects - TCPIP Demo App-C30\Delay.o
                  0x00b71e                  DelayMs
                  0x00b748                  Delay10us

MPFSHelpers       0x00b774          0xe
 MPFSHelpers      0x00b774          0xe Objects - TCPIP Demo App-C30\MPFSImg2-C30.o
                  0x00b774                  ReadProgramMemory

.isr              0x00b782          0x2
 .isr             0x00b782          0x2 default_isr
                  0x00b782                  _DefaultInterrupt
